:020000040800F2
:1030000000800020CBA900089D9E0008C19E0008FA
:1030100000000000000000000000000000000000B0
:103020000000000000000000000000005FAF00088A
:10303000000000000000000061AF0008FD0100205A
:103040009DA900089FA90008A1A90008A3A900083C
:10305000A5A90008A7A90008A9A90008ABA900080C
:10306000ADA9000805020020AFA90008B1A9000819
:1030700085020020B3A90008B5A90008B7A9000877
:10308000B9A90008ED9E0008FD9E00080D9F0008EC
:103090001D9F00082D9F00083D9F0008BBA9000848
:1030A000BDA90008BFA90008C1A90008E1020020CD
:1030B000C3A90008C5A90008C7A90008C9A9000834
:1030C000014802490160704708ED00E00030000847
:1030D000B0B51E4D2C1F20688006400F411E0329ED
:1030E00022D81B487944097949008F442301171AD3
:1030F000296803220A40032A00D016482968490695
:10310000490F491C07F062FA29684904490E4843EF
:103110002968490F491C07F059FA0BE07D2000028D
:1031200008E00120C00305E00C3D28688004410F41
:103130000848C84008490860226892093C231340A7
:10314000064AD258D0400860B0BDC0460C100240BC
:1031500000127A000024F4002004002060310008EE
:10316000000000000000000000000000000000005F
:10317000000000000000000000000000000000004F
:103180000100000002000000030000000400000035
:103190000600000007000000080000000900000011
:1031A000000000000000000000000000000000001F
:1031B0000100000002000000030000000400000005
:1031C00010B50124200208490A6802430A6002205F
:1031D00000F00CF8002801D0204610BD06F03EFE9D
:0C31E0000024204610BDC0460020024024
:1031EC00B0B505460E4801780124002916D07D2083
:1031FC00C00007F0E5F901460A48006807F0E0F95D
:10320C0000F0CAFD032D09D8002807D10024E043A3
:10321C002946224600F076FD034805602046B0BDE5
:0C322C00FA010020200400200C04002007
:103238000348007803490A68101808607047C046B8
:08324800FA01002068120020C9
:0C325000014800687047C046681200206A
:10325C00B0B50446FFF7F6FF0546601C02D00448E3
:10326C0000780419FFF7EEFF401BA042FAD3B0BD63
:04327C00FA01002033
:1032800003490A6802239A4302430A607047C04612
:0432900030000140C9
:1032940002480168012291430160704730000140F7
:1032A40003214902024A13688B43034313607047A6
:0432B40000000140D5
:1032B800F0B587B0044600200690002C60D0059039
:1032C800A06D002807D125465435204603F036FA6C
:1032D80000202870E06501273D072668B068C00017
:1032E80012D4B068814901402943B1608048006820
:1032F800804907F067F94000801C0690069800286E
:1033080002D00698401EF8E7B068284208D1A06DA0
:1033180010210143A165E06D012105910843E06595
:10332800B06804210140A06D102210404018A16D22
:1033380029D1204620300F230393DB430193F33B2D
:103348001940891CA165B168C90721D1F168182302
:103358009943A3680B43F36003218B0761680D460B
:103368001D40E76C2F43057F012D049313D1256C75
:103378002F43656C3D43A76C2F4301233B430BE070
:10338800012007B0F0BD1143A165384607B0F0BD74
:103398000021029118E03B463569574F2F400293B0
:1033A8001F4337610125EF07B9420DD0049B9942AD
:1033B8000AD0AB07994207D0039B9B0419404F4D95
:1033C8002F689F4379182960216B4B1E9941090387
:1033D800237E9B03657EEF031F43A57E6B033B4360
:1033E800E7681F430F4323690121002B00920491D2
:1033F80003DACA071946914300E049050F43017BE8
:1034080049003943007801280BD1002D029F0AD0CA
:10341800A06D20220243A265E06D01220243E2650D
:1034280003E0029F01E000040143039D606A002855
:1034380005D00722920110400843A16A0143F068B1
:103448002F4A02400A43F26030692E4A02403A434A
:103458003261706907229043626B0243726170693E
:1034680070229043A26B120102437261002B10D0AC
:103478000498400583421BD1206E00230246DA409F
:103488002A400F2A03D01B1D202BF7D106E0042B5E
:1034980004D1B06A019A1043B06209E0B26AE269E5
:1034A80092001C321C231340019A9A400243B262D4
:1034B800F068154A02408A420AD10020E065A06DF2
:1034C8000121014302208143A165059807B0F0BDA1
:1034D800A06D0099084302218843A065E06D049916
:1034E8000843E065084607B0F0BDC046E8FFFF6F37
:1034F80020040020400D030002FCFF1F08270140A4
:0C3508001902FEFF02FCFFDFE7FF3F831B
:1035140070B50546006881680024490701D4204637
:1035240070BD8168890704D481680F4A0A4010324B
:103534008260FFF78BFE0646286880684007EED558
:10354400FFF784FE811B28680329F6D381684907A5
:10355400F3D5A86D10210143A965E86D012420432A
:0C356400E865204670BDC046E8FFFF7F10
:1035700070B505460068816882680024D20726D0AD
:103580000222114023D1816805220A40012A16D166
:103590008168104A0A40911C816003210160FFF795
:1035A00057FE064628688068C00710D0FFF750FE17
:1035B000811B28680329F6D38168C907F3D0A86D59
:1035C00010210143A965E86D01242043E8652046E8
:0835D00070BDC046E8FFFF7F5B
:1035D800F0B581B005460024009400688168C907E9
:1035E8001AD18168214A2F32114208D0A86D1021C2
:1035F8000143A965E86D01242043E8650CE0816872
:103608001A4A1140012739438160194800680002AD
:1036180005D4687E01280FD1204601B0F0BD1548B9
:103628000068154906F0CEFF401C0090009800285D
:10363800EFD00098401EF8E7FFF706FE0646286818
:103648000168C907E8D18168C90704D18168074AB8
:10365800114039438160FFF7F7FD811B2868032972
:10366800EED30168C907EBD1C0E7C046E8FFFF7F8A
:0C3678000827014020040020400D030042
:10368400F0B581B00E46044601688B6802205B07E2
:103694001BD400925422A25C012A16D02746543728
:1036A40001253D70C868C0070AD18868C00704D0E6
:1036B4008868194A0240901C8860C8682843C8601A
:1036C4002046FFF787FF002801D001B0F0BDA06DB0
:1036D4001249014028020818A0650020E06521680D
:1036E4001C220A603870206D0D4A0E4B0E4DC562C7
:1036F400036342634A68102313434B6040313246EC
:10370400009B00F017FD21688A68034B13401A1DC3
:103714008A6001B0F0BDC046E8FFFF7FFEF0FFFF06
:0C372400DBA90008D1A900082DB10008A5
:10373000F0B589B0002508955422825C012A01D198
:103740000224DCE006465436012434700268936893
:103750005B0711D404694B68022B12D10420044387
:103760008148844252D17F48C0430B68D94301430A
:10377000906A084090624AE0816D20220A43826587
:10378000BCE00796069304263443764B764FBC4242
:103790004DD10F683B40906A1843906238025369DC
:1037A00083438968014071480840184350610024F0
:1037B000002F01D4079EA1E001266D483B46076813
:1037C00007208205394611406A48029383426CD132
:1037D000F0053B46034068D1654F3B68934319436E
:1037E0000143396066480068664906F0EFFE0C2127
:1037F00041430C31089108980028DBD0079E0898B7
:10380000401E089008980028F9D177E00B68002442
:10381000002B73D556480168574A934262D0574AE5
:10382000934262D0534A934268D105225BE00296EC
:1038300005951F27069C27400F2500950397BD403F
:10384000046E0195AC4304940F681F4246D0FB07F9
:10385000059D2C465BD1BB0754D47B0754D43B0752
:1038600054D4FB06344652D4BB0663D47B0663D4DF
:103870003B0663D4FB0563D40297BB0562D47B058A
:1038800062D43B0562D4FB0462D4BB0462D47B04E3
:1038900062D43B04009C3AD4FB035FD4BB035FD4E7
:1038A0007B03DB1712241C4031E03348029B834228
:1038B00003D130063B46034008D03048029B834288
:1038C00000D077E7B005074000D073E7284F3B688A
:1038D0009343194301433960079E0FE07B00DC0EE0
:1038E000059D14E00322920501E00322D205114058
:1038F00007229205036893435918016035702046EA
:1039000009B0F0BD012402E0022400E00324039E7C
:10391000B440049B1C430466069B9B08C069984204
:1039200000D83BE70198C043936A0340B800000FFA
:10393000B04031E70524EAE70624E8E70724E6E794
:103940000824E4E70924E2E70A24E0E70B24DEE7A1
:103950000C24DCE70D24DAE70E24D8E71024D6E7A0
:103960001124D4E7FFFF07000400008000FFFF07D9
:1039700008270140001000B0004000B8002000B44B
:0839800020040020400D0300AB
:10398800F0B582B05422825C012A01D1022159E1AA
:10399800026893685B07AE4E00D533E190C90839D9
:1039A800B44213D10124E505AF4260D00325AD052B
:1039B800AF4264D11F26B6068F683740D668A94B38
:1039C8003340A34EFB185B19D3605CE00126F30576
:1039D8009F425ED00325AB059F426AD11346A033B0
:1039E80000938B689E4F01931F409A4B9C426DD168
:1039F800002F00D199E0019CE30700D09DE0A307C8
:103A080000D5A3E0630700D5A1E0230700D5A2E015
:103A1800E30600D5A1E0A30600D5A2E0630600D521
:103A2800A3E0230600D5A4E0E30500D5A5E0A3059F
:103A380000D5A6E0630500D5A7E0230500D5A8E0DA
:103A4800E30400D5A9E0A30400D5AAE0630400D5E7
:103A5800ABE0230400D5ACE0E30300D5ADE0A3035D
:103A680000D5AEE06303DB1712261E40AAE0D36838
:103A780037467C4E1E4073193E46D36003E0D36838
:103A8800784D1D40D5602304846D9C438465802453
:103A9800AFE0714BDB43E5431D43E30C04261E40B6
:103AA8009319A0269F592F406C4D25403D439D51A9
:103AB8008EE0694BDB43E5431D43E30C04241C40C3
:103AC8001319A0241E592E401E5181E0002F30D01A
:103AD800019FFB0733D1BB07344631D47B0738D469
:103AE8003B072C462CD4FB0639D4BB063BD47B06BB
:103AF8003DD43B063FD4FB0541D4BB0543D47B05ED
:103B080045D43B0547D4FB0449D4BB044BD47B04C0
:103B18004DD43B044FD4FB0351D4BB0300D594E0F0
:103B28007B03DB1712241C400AE0019B5B00DE0EBE
:103B380048E0019B5B00DC0E02E0002642E0002426
:103B4800A640009C63683343636041E03AE0022684
:103B580038E00224F4E7032634E0042632E00424A3
:103B6800EEE705262EE00524EAE706262AE00624E5
:103B7800E6E7072626E00724E2E7082622E00824ED
:103B8800DEE709261EE00924DAE70A261AE00A24F5
:103B9800D6E70B2616E00B24D2E70C2612E00C24FD
:103BA800CEE70D260EE00D24CAE70E260AE00E2405
:103BB800C6E70F2606E00F24C2E7102602E010240D
:103BC800BEE711260123B340009D2C681C432C60DE
:103BD800846D0B681F4DAB421D4E05D101235D045A
:103BE800AC4384651C0204E001239D04AC43846556
:103BF8005C02146055680B7B012B01D1254300E062
:103C0800A543556054300D690C68B4420AD1D36895
:103C18009B08062633409D40D3689F0837404B6970
:103C2800BB4000E04B690021017028041843A3023F
:103C3800DC0F9B0F1B199B00D218136A0A4C1C40FF
:103C480004431462084602B0F0BD112478E7C04668
:103C58000000C07CFFFF1700FFFFC77CFFFF870045
:0C3C6800FFFF0700FFFF3F8300F000F0AB
:103C7400F0B583B00446002602965420205C012847
:103C840001D102253CE02746543701253D702046EA
:103C9400FFF76CFC21688A68D207A26D21D10090DD
:103CA40081235B009A43921CA265CA68CB680320F7
:103CB40001908343CB60EB078868184388600198C0
:103CC4000240114B886800280FD50298401C0290CE
:103CD40002989842F6D3A06D102202430220824338
:103CE4000CE010210A43054608E0C8681043C86088
:103CF400A06D0122024302208243009D3E70A26512
:0C3D0400284603B0F0BDC04600F20200EB
:103D1000002805D40322034693430C4A9A1806E070
:103D20000F220240083A03239A43074BD218800718
:103D3000C00E8901C9B28140FF23834010689843B7
:103D4000084310607047C0461CED00E000E400E04E
:103D5000002805D41F21084001218140014801604D
:083D60007047C04600E100E0DD
:103D6800002809D41F21084001218140034801602F
:103D7800BFF34F8FBFF36F8F7047C04680E100E0FD
:103D8800BFF34F8F034804490160BFF34F8F00BF53
:0C3D9800FDE7C0460CED00E00400FA0559
:103DA400401E010E01D0012070470749074A5060A8
:103DB400074803680B400321890759180160002054
:103DC4009060072111607047FFFFFF0010E000E0E2
:043DD40020ED00E0FE
:103DD800B0B50125002813D00446407F002803D140
:103DE8002077204602F02AFD0220607720790028FB
:103DF80008D0A168E268204600F026F8002808D01C
:103E08002846B0BD20680F49416181681822914356
:103E1800816000256079002801D0216900E0E9432C
:103E28002068016181686022914362690A43826067
:103E3800816880229143A2690A43826001206077E9
:083E48002846B0BDB71DC104FE
:103E5000F0B51F250024002D07D06D1E1F232B4019
:103E60000E46DE40F307F5D000E0E5430323164697
:103E7000DE410123032E0FD87E4436797600B74405
:103E800003010D100F2D07D80068416181681823C8
:103E900099431143816023461846F0BD072DF3D99D
:083EA000FAE7062DF0D9F7E75F
:103EA800F0B581B004464079012802D1022001B062
:103EB800F0BD15460E46022020710127677108687B
:103EC800042840D1002D08D02068406B002819D55F
:103ED800FFF7BAF90228F7D30CE00097FFF7B4F917
:103EE80007462068406B000414D5FFF7ADF9C01BE6
:103EF8000228F6D32069082101432161032020719B
:103F080001B0F0BD00970120FFF7A4F92068B1695E
:103F1800416405E00120FFF79DF92068B16901645B
:103F280010212940F2698A40214B8B40876C9F43BE
:103F380017438764326A8A40FF238B40C16C9943D8
:103F48001143C164009F2068316901290AD11021F9
:103F58000D407169A9401F22AA40836B93430B430C
:103F6800836301E010210D400721A940C26B8A43F9
:103F78003168B3680B43F1681943A9401143C16321
:103F8800B903A94002688A4302607168A940094AD6
:103F9800AA40036893430B430360C021A940026809
:103FA8008A43026000206071277101B0F0BDC046ED
:083FB800FF030000FE0F0000F2
:103FC000F0B583B0002840D00446064624360220CF
:103FD0007070276838683049014039602F48803058
:103FE000A0642F4838181425294606F0EFFA8000FF
:103FF0002A494118206401916164F8B208382946C1
:1040000006F0E4FA1F210140012528468840E064BB
:10401000A268E168114323690B4361691943A369ED
:104020000B43E1691943236A0B433968194339602B
:104030000295A9038A421B4A0AD1002301990B6009
:10404000636010601F461D461CE0012003B0F0BDF8
:1040500063683F211940019D29601060581E0023AC
:1040600003281F461D460DD8481E81005318002105
:10407000D96703210140029D8D400B4805607C33C8
:10408000BC3217460020E06323656765A565307084
:104090000299717003B0F0BD0F80FFFF000802406D
:0C40A000F8FFFDBF840802404409024004
:1040AC00F0B581B004462420205C012802D1022006
:1040BC0001B0F0BD25462435012028706E78012E04
:1040CC002CD1022068700020E06325682F680096D0
:1040DC00B7432F60A76CE66C7E60266D002E02D075
:1040EC00666DA76D7760266C1C273740009EBE401E
:1040FC000D4F3F6837430C4E37606B60A368102B35
:10410C00144600D00C46AC60102B00D01146E96070
:10411C002968009A1143296001B0F0BD0021297073
:0C412C008021E16301B0F0BD04000240FE
:10413800F0B582B004462420205C012802D1022078
:1041480002B0F0BD174625462435012028706A784C
:10415800012A2ED1022068700020E06325682A68B1
:1041680001260196B2432A60A26CE66C5660226D65
:104178000092002A02D0626DA66D5660226C1C2641
:104188001640019AB2401C4E366816431A4A166009
:104198006B60A368102B3A4600D00A46AA60102B21
:1041A80000D03946E9602968226B002A07D00E2220
:1041B8000AE0002129708021E16302B0F0BD0422E9
:1041C800914329602A680A2111432960019909024B
:1041D800626C1368DB0302D513680B431360009B02
:1041E800002B02D01A680A431A602968019A114301
:0C41F800296002B0F0BDC0460400024087
:1042040070B500282AD0014624314A78022A27D1E1
:10421400046822680E239A432260426C1568134B8B
:104224001D4015602568012295432560046C1C25FA
:1042340025401446AC400E4D2E6826432E60846CF7
:10424400C56C6560046D002C05D025681D40256093
:10425400436D806D58604A70002004E0012070BDF9
:104264000422C263012000220A7070BDFFFEFFFF1A
:044274000400024000
:10427800F0B585B00446054624356878022809D18A
:104288002068006880060CD41646002901910DD0DC
:1042980004220CE0002028700420E063012005B00F
:1042A800F0BD01200102E16305B0F0BD0222206CDF
:1042B8001C2104910840824003923348071FFEF7EF
:1042C800C3FF039A02903868104217D1216C0498F2
:1042D80001403868C840000748D4701CF3D0FEF786
:1042E800B3FF039A002E03D00299401AB042EAD9CC
:1042F8002020E06300202870012041E0206D002884
:104308000ED0616DA26D0B681A4209D001231E02FE
:104318000768374307604A609802E16B0143E1632D
:10432800A06CE16C0268114205D041600120400296
:10433800E16B0143E163206C04990840019900296D
:1043480008D004218140104A1068084310600020FA
:1043580005B0F0BD022181400B4A10680843106087
:10436800002028700121697005B0F0BD01200246C7
:104378008A40054B196811431960E06300212970D0
:0C438800687005B0F0BDC04604000240A3
:10439400F0B585B00E46234D2978012902D10220BB
:1043A40005B0F0BD17460193049000246C60012011
:1043B400039028707D20C000029000F037F8002898
:1043C4002DD10399029B0094174D0498012809D11B
:1043D4002868084328603760BFF36F8F01987060C6
:1043E400184614E08804296801432960EFF3108417
:1043F40072B6009904CF04C64A1C3F291146F9D36A
:104404001846291F0968C903FBD484F3108800F0F7
:104414000DF82968049A91432960024D009C2C7080
:0C44240005B0F0BDD811002014200240AB
:1044300070B50446FEF70CFF0619104D2868C0033E
:1044400005D5FEF705FFB042F8D3032070BD2868FC
:104450000B494A1C2A60084003D00A4948600120E1
:1044600070BDFEF7F5FE04192868400304D5FEF779
:10447000EFFEA042F8D3E8E7002070BD1020024014
:08448000FAC30000D81100206E
:104488000648C168002901D400207047044901602A
:1044980004490160C068C00F7047C0460820024048
:0844A80023016745AB89EFCD4C
:1044B0000120C00703490A6802430A600868C04334
:0844C000C00F704714200240F8
:1044C800F0B583B00546284C2078012802D1022097
:1044D80003B0F0BD029100276760012020707D20A5
:1044E800C6003046FFF7A0FF002839D104206860D5
:1044F8002868042809D11E48801C1C490A68024300
:104508000A603046FFF790FF2AE0F84302990860F6
:104518003946AF68E868C01987420191084619D240
:10452800FC0012490868134A10402043104A1043FF
:1045380008603046FFF778FF002808D1A868E968C6
:10454800081808347F1C8742EBD3019801E00299D0
:104558000F60054C054B1968022291431960019FB1
:10456800277003B0F0BDC046D811002014200240C7
:084578000200010005FEFEFF38
:10458000F0B58AB00C68002C00D1C3E00246624846
:10459000824201D0052000E00320009000231E4647
:1045A000099308930691049211E03043079E5B4CF7
:1045B00060605B1C0C682046D840089D2D1D089546
:1045C0000836099DAD1C0995002800D1A2E00125FF
:1045D00003959D402C400594EBD0099A07964F68AF
:1045E000032408463E462640711E0129029714D82E
:1045F000019313469440049A9168A143C06898407F
:1046000008439060F806019BC00F98405168A94389
:1046100001435160E5435F000AE0204617469040A1
:10462000C543032E049A03D109982646044623E085
:10463000D06828401446069A9168B9400143E16069
:10464000022E3C4617D11C20089908400F218140BA
:104650000294DC08A400049F3C192E46256A8D4371
:1046600011698140294335462162029C5168032625
:104670000E403A4601E0049A0299A640106828408C
:10468000304310608803800F0699079E91D018214F
:1046900031400F20884003241D46A5431F4C661956
:1046A000356E854360360520000782420CD01D48D8
:1046B000824206D01C4882420098194A06D1022044
:1046C00004E0174A039801E00020154A8840284377
:1046D0003060106806994D68EC0302D5059E3043A2
:1046E00001E0059EB04310605068AC0301D5304333
:1046F00000E0B043506009480068EC0201D5304347
:1047000000E0B043054A10605068AA0200D54CE7AB
:10471000B0434BE70AB0F0BD000C00500018024057
:0C47200080180240000400500008005007
:10472C00F0B58AB00290002973D03B48029A8242BD
:10473C0001D0052000E003200090002422462746EB
:10474C002646019125E0069D099885400868284376
:10475C0008601C20089C2040059B8340F0088000CA
:10476C0008180A46016A994301629068A843906050
:10477C005068079988435060D068A843D060099A64
:10478C000199761C0846F040241D921C083700281D
:10479C003FD001231846B04005460D40F1D007909C
:1047AC000992089418243C400F2005900146A14022
:1047BC000320324606908243184880180390026EFC
:1047CC0004910A40052000070299814208D015483F
:1047DC00814206D014488142009B02D1022300E0A2
:1047EC000023A3409A42AED1039B60330C4A10685D
:1047FC00A84310605068A8435060084A1068A8434A
:10480C0010605068A84350601868049A9043186070
:10481C0099E70AB0F0BDC046000C005000180240E9
:0C482C00801802400004005000080050FA
:10483800F0B581B0032569020F4E32688A430243FE
:10484800326001214A020024904212D10B480268CA
:10485800706940050DD58F0206205043084905F0C0
:10486800B1FE801C401E03D071693942FAD100E0C4
:104878002C46204601B0F0BD007000402004002006
:0448880040420F009B
:10488C00F0B587B00125002800D1EFE10495059023
:10489C000078C007FD4F2AD0B868F96803252A466E
:1048AC008A43382101401020484082185042504120
:1048BC00082914D0002812D105984268012001045F
:1048CC008A4208D005231B049A4200D028E18204B6
:1048DC003B6813433B603A680A433A6029E1386805
:1048EC00800304D505984068002800D188E005981D
:1048FC00007880073CD405980078000768D4059AA6
:10490C001078400771D4D06900282FD0B9683822AC
:10491C000A40102A00D0DBE0012871D0F86803218E
:10492C000140059B1A6A91426AD1702101405A6A72
:10493C00914265D17F21090201409A6A120291428B
:10494C005ED11F2149040140DA6A914258D10721F6
:10495C004A0602401C461B6B9A42049D00D085E11E
:10496C0049070840616B884200D07FE100257DE15A
:10497C00B9683820084010214140FA6803263240BB
:10498C0002235340CA18514251410125AC02002860
:10499C0038D0002936D13868059AD168002900D161
:1049AC00D5E00721C9028843116901433960280207
:1049BC00396801433960FEF745FC054638682042EA
:1049CC0000D0D5E0FEF73EFC401B0228F6D9CDE026
:1049DC00B8683821014018293CD1386E80078ED533
:1049EC000598806900288AD10AE0B868382101400E
:1049FC00202946D1F86D800785D59068002882D192
:104A0C00049D33E139682142059B03D0D968002904
:104A1C0000D12BE17F2109027A688A435969090286
:104A2C001143796000280DD10720C00239688143F9
:104A3C0018690843386038688004400F9949C140B0
:104A4C009948016099480068FEF7CAFB002800D01D
:104A5C000CE150E7386E05998969002900D1A7E06F
:104A6C00012108433866FEF7EDFB0646386E8007D9
:104A7C0000D544E7FEF7E6FB801B03250228F5D999
:104A8C00F4E0012003900107F86B0840029006D176
:104A9C00F86B0843F863F86B084006900698019190
:104AAC0083480068C0052AD403980402804908682A
:104ABC0020430860FEF7C6FB06467D48006820428E
:104ACC001DD1FEF7BFFB801B03250228F5D9CDE0D5
:104ADC0001221306396899433960022852D1039395
:104AEC0004925406FEF7AEFB0646386820427ED090
:104AFC00FEF7A8FB801B03250228F6D9B6E0059823
:104B0C0080686C4C012806D0052800D098E0F86D20
:104B1C0004210143F965F86D03990843F86599E0A0
:104B2C003B688B433B6081043B688B433B60002AB2
:104B3C004FD04404FEF786FB06463868204200D06E
:104B4C00D5E6FEF77FFB801B6428F6D98EE02902A0
:104B5C0088433860FEF776FB05463868204200D162
:104B6C00C9E6FEF76FFB401B0228F6D935467DE0FF
:104B7C007F20000279688143059840690002084350
:104B8C007860B8E6F8680325A843F860F8684A49E5
:104B9C000140F9605606FEF755FB04463868304272
:104BAC0000D1E3E6FEF74EFB001B0228F6D95DE0D0
:104BBC00012188433866FEF745FB0646386E8007B0
:104BCC0000D49CE6FEF73EFB801B03250228F5D99A
:104BDC004CE04404FEF736FB06463868204200D110
:104BEC0085E6FEF72FFB801B6428F6D93EE0F868BB
:104BFC0032490140059A106A0843516A0143906A90
:104C0C0000020843D16A0143106B526B08431043F6
:104C1C00F860386803990843386004980007F9680D
:104C2C000143F960FEF70EFB06463868204200D0BF
:104C3C009CE6FEF707FB801B03250228F5D915E03F
:104C4C00F96D039A9143F965F96D04229143F96565
:104C5C0000280ED0FEF7F6FA0646F86D800717D43A
:104C6C00FEF7F0FA801B0325A042F6D9284607B0C0
:104C7C00F0BDFEF7E7FA0646F86D800708D5FEF79B
:104C8C00E1FA801B0325A042F6D9EFE700100240A1
:104C9C0002980028059A00D035E6F86B01998843F4
:104CAC00F86330E60024F400200400200C040020FB
:104CBC000070004088130000FFFFFEEE8C80C111D5
:104CCC00F0B583B00D460121002800D1A3E001917D
:104CDC0002905248006807242040A84213D24F4942
:104CEC000868A043284308604D4EFEF7ABFA074610
:104CFC004A4800682040A84205D0FEF7A3FAC01B22
:104D0C00B042F5D986E0029B18688107454E0CD558
:104D1C00410703D5210332680A4332600F2109028F
:104D2C0032688A43996811433160C00718D13B48F7
:104D3C0000682040A84228D938490868A043284375
:104D4C000860374FFEF77EFA06463448006820406C
:104D5C00A8421AD0FEF776FA801BB842F5D959E072
:104D6C00586803282FD8810001A2515832468F462B
:104D7C008D4D0008D94D0008E34D0008ED4D00089D
:104D8C0011460839096849052CE0029A1078400749
:104D9C00244D05D5200329688143D0680843286039
:104DAC0000F048F8296889093C220A401E498958B4
:104DBC001F220A40D0401D4908601D480068FEF7BC
:104DCC000FFA014627E03246516D0AE011460839C8
:104DDC000968890306E0114608390968890101E070
:104DEC00916D8907019916D51168A1430143116092
:104DFC000B4FFEF727FA06460A4800683821014097
:104E0C0002984068C000814291D0FEF71BFA801BCB
:104E1C00B842F1D90321084603B0F0BD002002408E
:104E2C0088130000081002406031000820040020A4
:044E3C000C04002042
:104E400010B51E4C20688006400F06D0206838211F
:104E5000084008281A4807D110BD083C2068800483
:104E6000410F1848C84010BD22680A40102A15D1C9
:104E7000616803220A40032A00D01248616849068B
:104E8000490F491C05F0A2FB61684904490E4843DB
:104E90006168490F491C05F099FB10BD2068084066
:104EA000202802D10120C00310BD20680840182826
:104EB00001D0002010BD7D20000210BD081002406E
:084EC00000127A000024F40046
:104EC8000648006806490968890A1C220A400549FB
:104ED80089581F220A40D0407047C046200400204D
:084EE80008100240A03100088F
:104EF0000120C00402490A6802430A607047C046A4
:044F0000001002405B
:104F040010B50320000208490C6820404860E00501
:104F140002D4A00504D410BD05F0FEFDA005FAD509
:0C4F240005F0FBFD10BDC0461C10024053
:104F3000F0B587B0817889077A4F01D400264EE01A
:104F40000590012319073A46183A10680840049062
:104F500006D1106808431060106808400690069853
:104F60000292039101931E026F4C2068304320602F
:104F7000FEF76EF905462068304207D1FEF768F962
:104F8000401B0228F7D90326059820E00320054698
:104F90000102B868084012D00599096B88420BD00D
:104FA000B86801990904BA680A43BA60BA688A43C2
:104FB000BA605E490840B860C00700D0A1E0BA6896
:104FC0005A4802400598016B1143B96000260499C4
:104FD000002904D1029B1968039A9143196005685E
:104FE000E90762D1A90768D4E9066ED4A90575D48A
:104FF00069057CD4A90606D5032109033A688A43CA
:1050000001691143396001216A040ED53A68494BA0
:105010001A40046A22433A605A1C944205D10A0499
:105020003B46483B1C6814431C602A0305D53A687C
:1050300040239A43436A13433B608A05AB0211D570
:105040003B689343846A23433B6094420AD10B0636
:1050500004933C46483C0590304626681E43266033
:105060000646059815420CD00A063B689343C46A6D
:1050700023433B60944204D13B46483B1C681443A5
:105080001C602A050ED58C03032292033B689343D0
:10509000426913433B60A24204D10804483F396887
:1050A00001433960304607B0F0BD396803229143AF
:1050B00042680A433A60A90796D539680C229143A1
:1050C00082680A433A60E90690D5032189023A686A
:1050D0008A43C16811433960A90589D50321890430
:1050E0003A688A43816911433960690582D5032191
:1050F00009053A688A43C16911433960A90682D516
:105100007AE7FEF7A5F80646094CB868800700D58F
:1051100055E7FEF79DF8801BA042F6D905982E466C
:1051200055E7C0465410024000700040FFFCFFFFEE
:0851300088130000FFFFFF3FA0
:1051380030B5056801229407A04205D0234B984258
:1051480002D0234B984204D170239D434B682B43D4
:1051580000E02B461F4DA84209DD1F4CA0420FDC82
:105168001A4CA04212D01F4CA0420FD02BE0A042F4
:105178000CD0174CA04209D01B4CA04206D022E00C
:10518800164CA04202D0164CA0421CD10324240283
:10519800A343CC681C4380239C434B69234303608F
:1051A8008B68C3620B688362104BC3180A24E341FF
:1051B800072B06D814469C40E1231C4201D00969FC
:1051C8000163426130BD1C46E5E7C046002C014042
:1051D80000040040FF2B0140FF430140004801400C
:1051E80000440140004001400020004000D4FEBFC0
:1051F8003D21415C01290FD101463D3102220A704F
:1052080001681148814209DC0120800781420BD0E6
:105218001048814208D011E0012070470B488142B4
:1052280002D00B48814209D188680B4A024000200D
:10523800062A08D001231B049A4204D008680122D8
:1052480002430A6000207047FF2B014000400140E4
:0C525800002C0140000400400700010091
:1052640010B53D21415C012912D101463D31022294
:105274000A700168C86801221043C8600F4881425F
:1052840008DC900781420BD00F48814208D010E01F
:10529400012010BD0A48814202D00A48814208D147
:1052A40088680A4B03400020062B06D01404A3424E
:1052B40003D0086810430860002010BDFF2B014094
:1052C40000400140002C01400004004007000100A0
:1052D40010B50268D36801218B43D360136A074C6D
:1052E400234206D1136A064C234202D113688B432E
:1052F40013603D228154002010BDC04611110000EE
:04530400440400005D
:10530800B0B50446006801698907554D17D5C168CD
:10531800890714D52946FE31016101212177806969
:10532800800703D0204605F022FC05E0204605F062
:105338001FFC204605F01DFC00202077206801692D
:10534800490718D5C168490715D52946FC310161B7
:105358000221217780698005800F03D0204605F05F
:1053680006FC05E0204605F003FC204605F001FC9C
:105378000020207720680169090717D5C168090747
:1053880014D52946F831016104212177C0698007C5
:1053980003D0204605F0EBFB05E0204605F0E8FBCE
:1053A800204605F0E6FB0020207720680169C90641
:1053B80018D5C168C90615D52946F03101610821FB
:1053C8002177C0698005800F03D0204605F0CFFB08
:1053D80005E0204605F0CCFB204605F0CAFB00207E
:1053E800207720680169C90709D0C168C90706D0B4
:1053F8002946FF310161204604F0A4FD20680169B7
:10540800090609D5C168090606D529468031016112
:10541800204605F0B1FB20680169C90507D5C168B8
:10542800090604D50561204605F0A7FB2068016937
:10543800490609D5C168490606D52946C031016122
:10544800204605F097FB20680169890607D5C168E1
:10545800890604D5E0350561204605F08CFBB0BD12
:04546800FFFEFFFF45
:10546C0070B53C22825C012A01D1022070BD02463B
:10547C003C320223537000688368474C1C408460A4
:10548C000B683F2B19DD5F2B1EDD602B41D00124F7
:10549C006503AB4255D0702B79D1FF231B02846876
:1054AC009C434B688D68C9681D43090229432143FD
:1054BC00816083687721194368E01F2B1EDC002B69
:1054CC0020D0102B1ED062E0402B4AD0502B5ED146
:1054DC00036A046A0125AC4304628469F025AC4379
:1054EC00CD682D01254385610A24A34349681943DE
:1054FC000162836829491940573147E0202B01D0BC
:10550C00302B44D18168254C0C402343072119438F
:10551C003CE0036A1024A34303620F231B0384693A
:10552C009C43CB681B032343046A8361A0239C43E5
:10553C0049680901214301628368184919406731A0
:10554C0024E0FF231B0285689D434B688E68C96865
:10555C001E430902314329438160A3038168194327
:10556C0014E0036A046A0125AC4304628469F025E3
:10557C00AC43CD682D01254385610A24A3434968BA
:10558C001943016283680549194047318160002045
:10559C0010700121517070BD8800CEFF88FFCFFFC5
:1055AC0070B53C22825C012A01D1022070BD0246FA
:1055BC003C3202235370006845688368134CA04248
:1055CC0001D02E4604E00F263605B5434E682E4317
:1055DC007025AE430D68354345600D4DA84205DC82
:1055EC000124A407A04206D00B4C02E0094DA842AE
:1055FC0001D0A04204D18024A3438968194381605F
:10560C00002010700121517070BDC046002C01406B
:0C561C00FF2B0140004001400004004052
:10562800F0B581B004460268106871490140A0686D
:105638002369034360691843E3691843084310600A
:105648000327380351688143E06808435060A16923
:10565800684DAA4202D0206A084300E008469168D3
:10566800654E0E4006439660D06A0F218843616AF2
:105678000843D0620026614882420EDD60488242BB
:105688001DD0AA4211D05F4882420CD16048006800
:105698008007000F5F4E365811E05B48824208D001
:1056A8005A4882420BD0102609E059480068000A7F
:1056B80001E0574800680C2606405648865920469F
:1056C800683000905448AA4214D00125EA03934256
:1056D80022D1082E00D981E07E4436797600B7447D
:1056E800047D547D4D7D7D7D5300FFF7E9FB002847
:1056F80048D172E00125082E00D96FE07E44367942
:105708007600B744046B216B196B6B6B1F00FFF7B6
:10571800D7FB002814D160E0082E5FD87E44367984
:105728007600B744045B4B5B445B5B5B4A00FFF766
:10573800C7FB00283FD150E0FFF77EFB00284CD084
:10574800616A01E00120C0034900344A515A04F05B
:1057580039FF62685743B84240D3110388423DD8A5
:10576800010E5608000200238019594104F04EFF2B
:105778002C4941182C4A91422DD32FE0FFF75CFBAE
:1057880000282AD0616A00E010464900234A515A8D
:1057980004F018FF400061684A08101804F012FF6E
:1057A8001F4901401AD00007400F084313E0FFF7D4
:1057B80043FB002811D0616A00E010464900174AEF
:1057C800515A04F0FFFE61684A08101804F0FAFE06
:1057D80080B2102802D32168C860002513480099B8
:1057E8000860002020676067284601B0F0BDC04609
:1057F800F369FFCF00800040FFF4FF11FF4B00402A
:10580800004C00400038014000440040004800407F
:1058180054100240F0A800080024F400C4B30008A3
:10582800F0FF000000FDFFFF00FD0F000100010078
:10583800F0B581B00546074680370024FC60FDF7C7
:1058480003FD06462868016809070BD51148009032
:105858000120410500222846334605F0F8F90028C2
:105868000ED12868006840070CD50A48009001202E
:10587800810500222846334605F0E9F9002801D0C1
:10588800032404E020207860B8603C70EC66204671
:0858980001B0F0BDFFFFFF01AC
:1058A000F0B581B0054604468034606802232028A4
:1058B00011D10120002950D0002A4ED0AE680090AE
:1058C0000703BE420AD1C80708D02869002805D1BD
:1058D000009801B0F0BD184601B0F0BD2078012855
:1058E00018463AD02B4654335A800020E0601A8084
:1058F000296521216160009B59076A6E8A4206D1A1
:10590000BE4202D12869002808D0184907E0BE42EB
:1059100002D12969002912D0124911E01249002050
:1059200020706967EFF3108183F31088DA052B6824
:105930009C6814439C6081F3108801B0F0BD084955
:1059400020706967EFF3108183F310882A68136869
:1059500080241C43146081F3108801B0F0BDC04660
:10596000E959000869B2000871590008FDB1000842
:1059700070B58421415821291AD1014656318A8AAD
:10598000002A15D0174B02E0521E140410D00C88C8
:10599000002C0ED00468E5692D06F5D5056D2E881E
:1059A0001E40A662AC1C04650C88641E0C80EBE7EC
:1059B00070BDEFF31081012282F31088D3050468D3
:1059C000A5689D43A56081F31088EFF3108182F3F1
:1059D00010880068026840231343036081F3108835
:0859E00070BDC046FF0100008C
:1059E80030B58421415821290FD1014656310A8802
:1059F800002A0BD0026D1388104C1C4003689C626F
:105A0800921C02650888401E088030BDEFF31081A3
:105A1800012282F3108803681C688025AC431C604F
:105A280081F31088EFF3108182F310880068026810
:105A380040231343036081F3108830BDFF01000049
:105A4800F0B581B0034680339C680226202C10D123
:105A5800012400290ED0002A0CD001252C038768C8
:105A6800A7420AD1CC0708D00469002C05D12C46DE
:105A780000E03446204601B0F0BD1C78012C3446C5
:105A8800F8D00024C4661D7003680A4EB3420DD0D6
:105A98005B681B020AD5EFF3108385F31088AD0607
:105AA800066837682F43376083F3108800F004F8DE
:085AB800E0E7C0460080004059
:105AC000F0B582B05C23C2528165002101670446B3
:105AD0005C346280856803468033002D0BD001263C
:105AE0003707BD420CD03603B5420ED10569002DF3
:105AF00004D1334D0CE00569002D08D1FF2507E0E6
:105B00000569002D03D03F2502E0A18001E07F253B
:105B1000A5800191D96022259D60EFF310860125B3
:105B200085F310880768B9682943B96086F310883F
:105B3000290200912F036907466E8E4202D1A18986
:105B4000914216D98168B94202D10169002933D046
:105B50001F4A0199009C19700267EFF3108185F3C9
:105B600010882034006802682243026081F31088A4
:105B70001FE08168B94202D1016900291ED0124A92
:105B80000199009C19700267EFF3108185F310886A
:105B9000026813682343136081F31088EFF31081C8
:105BA00085F310882A07006883681343836081F3B4
:105BB0001088002002B0F0BD044ACAE7014ADFE7BE
:105BC000FF010000D55B0008715D0008C1B200084C
:045BD0004DAD0008CF
:105BD400F0B585B004460168C8690D688B6826462F
:105BE4005C36B788F26A222A00D093E0039320211E
:105BF4000191B189002900D192E00199084000D1B6
:105C04008EE00121184608400390049108020540E3
:105C14000095029707E0204605F095F8009DB80628
:105C2400029F00D47CE02068416A3940A26D118053
:105C34007188491E7180911CA165C769790732D0AA
:105C44006A426A41FB07049B00D01346002B04D12F
:105C540001220262336B13433363039B5A425A415A
:105C6400BB07049B00D51346002B05D10222026218
:105C7400326B042313433363039B5A425A41002972
:105C8400049900D51146002905D104210162306B25
:105C9400022101433163306B002804D0204605F013
:105CA4004FF80020306370880028B8D1EFF31081DA
:105CB400012080F31088020223681D6895431D604B
:105CC40081F31088EFF3108180F3108822689368C1
:105CD400244D2B40936081F310880199F1620021D7
:105CE4002167E26E012A96D1E166EFF3108180F319
:105CF40010882268136810208343136081F310888E
:105D04002168CA69D20600D508623188204605F0A8
:105D140018F883E78869082202438A6105B0F0BD58
:105D240070880028FAD0B1898842F7D2EFF3108046
:105D3400012181F310880B4A521C23689D68154089
:105D44009D6080F3108808482067EFF3108081F38A
:105D5400108821680A68019B1A430A6080F310883E
:0C5D640005B0F0BDFEFFFFEFC1B200086B
:105D7000F0B585B004460168C8690D688B68264691
:105D80005C36B788F26A222A00D095E0039320217E
:105D90000191B189002900D194E00199084000D116
:105DA00090E0012118460840039004910802054044
:105DB0000095029707E0204604F0C7FF009DB80653
:105DC000029F00D47EE02068406A3840A16D0870D0
:105DD0007088401E7080A06D401CA0652068C76957
:105DE000790732D06A426A41FB07049B00D0134610
:105DF000002B04D101220262336B13433363039BF4
:105E00005A425A41BB07049B00D51346002B05D1CB
:105E100002220262326B042313433363039B5A4210
:105E20005A410029049900D51146002905D10421C1
:105E30000162306B022101433163306B002804D0D2
:105E4000204604F07FFF0020306370880028B6D120
:105E5000EFF31081012080F31088020223681D688F
:105E600095431D6081F31088EFF3108180F3108853
:105E700022689368244D2B40936081F31088019928
:105E8000F16200212167E26E012A94D1E166EFF30D
:105E9000108180F3108822681368102083431360F8
:105EA00081F310882168CA69D20600D5086231885A
:105EB000204604F048FF81E78869082202438A618E
:105EC00005B0F0BD70880028FAD0B1898842F7D2B9
:105ED000EFF31080012181F310880B4A521C2368D4
:105EE0009D6815409D6080F3108808482067EFF397
:105EF000108081F3108821680A68019B1A430A60A8
:105F000080F3108805B0F0BDFEFFFFEF4DAD000837
:105F1000F0B581B000283AD016460F4604460093EB
:105F2000054680356868002803D12870204604F0B3
:105F3000ABFA24206860206801680125A94301604C
:105F40002046FFF771FB012822D0A06A002802D06A
:105F5000204604F017FE0120820321688B6813435A
:105F60008B60C2038B6893433B438B607205009B3D
:105F70001B0413430A68084D15401D430D600A6851
:105F800002430A602046FFF757FC054600E0012562
:0C5F9000284601B0F0BDC046FFFF00FC39
:105F9C00F0B581B0054668352A7E012A02D102206F
:105FAC0001B0F0BD2422EA6106683768326801242A
:105FBC00A243326007225207B36893430B43B3608A
:105FCC00406E0028204615D00097B768B068400F87
:105FDC000D49095C0D4A105CC00004F0F1FA04464E
:105FEC003801009F400F0849095C084A105CC0004A
:105FFC0004F0E6FA28806C80376000202876202197
:10600C00E96101B0F0BDC04659BB000851BB0008A6
:10601C00F0B581B0054668352A7E012A02D10220EE
:10602C0001B0F0BD2422EA610668376832680124A9
:10603C00A243326007225206B36893430B43B3600A
:10604C00406E0028204615D00097B768B068400F06
:10605C000D49095C0D4A105CC00004F0B1FA04460D
:10606C003801009F400F0849095C084A105CC000C9
:10607C0004F0A6FA28806C80376000202876202156
:10608C00E96101B0F0BDC04659BB000851BB000826
:10609C00F0B5FFB0FFB095B0FFAD3C3508920E46A1
:1060AC0003905449694408600021534868440160D6
:1060BC000EA8E96028600124A0026860C84305901E
:1060CC0009940C9508E02B4600F032FAA1E0099CEB
:1060DC00E968002900D526E20D913178761C252936
:1060EC000BD0002900D103E26A68AB68581C9042BF
:1060FC0028D918469042EBD12DE000273078024683
:10610C00233A0D2A14D802217A441279520097446A
:10611C000B0F0F0F0F0F0F0F0D0F090F0F060F4364
:10612C00761CEBE72146FAE70821F8E70421F6E7AD
:10613C000921C94302463A3A00258A4216D22C4616
:10614C00324620E02A68D154A860E968491CE9600D
:10615C006A689042BCD12968286904F08BFBA96855
:10616C00884200D0D4E10020A860B1E700240A23C3
:10617C005C432418303C721CDB43707806463A3E74
:10618C009E421646F3D82E2814D1501C5278134632
:10619C003A3B8B4201D206460CE000250A214D43C6
:1061AC00AD18303D461CC943427810463A388842F7
:1061BC003046F3D83078FB210140761C6829F9D0A1
:1061CC0001465839202931D87944097949008F443E
:1061DC0022202020202020202020203B472020206F
:1061EC002020202020202020682020752015202011
:1061FC002200C0464804000040040000089A1068C1
:10620C00011D1160016800940197FFA83C300A221F
:10621C0059E70C9D5BE7089A1068011D1160016835
:10622C0000940197FFA83C3010224CE72528F0D1B0
:10623C000C9D6A68A968481C9042099C7ED9084646
:10624C00904200D044E786E708990B68181D086057
:10625C000C9D6A68A968481C904260D9084666E0A3
:10626C00089A1068011D11600168C8170691414019
:10627C00081A01220A2809D30B920A210A9004F069
:10628C009FF90B9A521C0A996329F5D8AA4200D897
:10629C002A46002C0D994FD00698002852D4002085
:1062AC0051E0089A1068011D116001680020082354
:1062BC0000930190FFA83C30102205E7089A106863
:1062CC00011D116005680C998868CC6804E038469B
:1062DC006D1C0D9100291ED4297800291BD0471C58
:1062EC000C9B5A68974204D907460D999742EED1F8
:1062FC0006E01A681154641C5A6821469742E6D18C
:10630C000C980168006904F0B5FAB84200D0FCE0C2
:10631C0000202146DCE70C9DA860EC60D7E61A68EB
:10632C002B685A54A860E968491CE9606A68099CA2
:10633C00904200D0CCE60EE700230AE02A68252321
:10634C00535401E701200421394089080143631AA1
:10635C000D99022038400490099C0B9201D0002D1D
:10636C003ED0F8073CD1002B3AD00C9988680A90A3
:10637C00C96807910D9806E00A9400280D9B099CAA
:10638C000B9A00D59EE0591E0D91994221D29A424A
:10639C001FD20A994C1C0C9B5A68944203D90C4688
:1063AC009442E9D109E00846196820220A5407985A
:1063BC00401C5A6807909442DED10C980168006921
:1063CC0004F058FAA04200D0A5E000200A900798EB
:1063DC00D3E702460C990A9888600798C860114662
:1063EC0000296DD40698002804D4780729D50D917E
:1063FC002B2103E00D91404206902D210A930C9C19
:10640C006268A368581C904202D918460D9906E0A0
:10641C002268D154A060E168491CE1606268099C63
:10642C0090420BD10C9C2168206904F023FAA168DE
:10643C0088426DD10020A060E168099C00290A9B6C
:10644C003ED40498002848D001203840284344D139
:10645C00002B42D00A460C99486804908868C96899
:10646C00079111460B9A05E0204600290A9B099CCE
:10647C000B9A28D40D90581E0A90984228D29A4212
:10648C0026D20B460D98441C0C994A68944204D9A8
:10649C00044619469442E7D108E0096830220A54B0
:1064AC000799491C0791049A9442DDD10C98016814
:1064BC00006904F0DFF9A0422DD100200799D4E740
:1064CC000C9D05E60A980C9DA8600798E860FFE50E
:1064DC000C9A0D9890600798D060069900930197DC
:1064EC00FFA83C300A222B4600F022F80C9DEFE569
:1064FC000D9900290ED0AA68002A12D00EA9039873
:10650C0004F0B8F9A868E9680CE00C988760C460DE
:10651C00059908E007E00C9884600799C16005991B
:10652C0001E00020091808467FB07FB015B0F0BD1F
:10653C00F0B585B001930290012403919142264657
:10654C00049207D30846114604F03AF8049A761CD4
:10655C009042F8D20B980A9A01998E4200D80E46B6
:10656C000440002A009419D0002C17D12021800758
:10657C0001D40F4600E030270198002800D00F46C8
:10658C00029C002A0AD0964208D22046394615466B
:10659C0004F0E0FE6A1EE0680028F2D50298C0689C
:1065AC00002840D40124019F02E07F1E04994C4333
:1065BC00022FFAD203982146154604F001F82A4618
:1065CC0004998842F3D20196039E039630462146E5
:1065DC0003F0F6FF07461548C15D029E304604F0F5
:1065EC00B9FEF068039E002809D46743F61B2046C9
:1065FC00049F394603F0E4FFBC420446E5D2009800
:10660C000028019E0FD0002D0DD06C1EAC420AD27A
:10661C00AE4208D22021029D284604F09BFEE86879
:10662C0000282546F1D505B0F0BDC04661BB000879
:10663C0070B584B03C213848002545542C210126E6
:10664C004654C56402218163466345628562062116
:10665C00C161867605830824304932030263021D2A
:10666C00157701607105B20742608560C5600161F4
:10667C004461039502950195FCF718FE002801D0A2
:10668C0002F0A0FA2648039002950196224801A92F
:10669C00FDF748F8002801D002F094FA0395042085
:1066AC000290204801901C4801A9FDF73BF80028F6
:1066BC0001D002F087FA02941B480190164801A9F8
:1066CC00FDF730F8002801D002F07CFA0C20029083
:1066DC0016480190104801A9FDF724F8002801D0B4
:1066EC0002F070FA10200290114801900A4801A99A
:1066FC00FDF718F8002801D002F064FA142002907B
:10670C000C480190044801A9FDF70CF8002801D0B1
:10671C0002F058FA04B070BD840E00200024014031
:10672C0004FFFF0702000004040000080800000C2E
:08673C008000001C4000001861
:10674400F0B595B0044600261496139603A8001DD0
:10675400302103F0C1FF20682749884201D015B0D9
:10676400F0BD01940127B803039003A8FEF7DEFBF4
:10677400002801D002F02AFA38052049CA680243E9
:10678400CA60CA68024002920298086838430860E6
:106794000868384002901296CF2010900298032582
:1067A40011950524200710A9FDF7E8FE2803144DD0
:1067B40028622020B9023A028023124F2F606C60B5
:1067C400AE60EE602B616A61A961E8612846FDF75D
:1067D400F5FB002801D002F0F9F90198A8620565DB
:1067E4000C24002120460A46FDF790FA2046FDF7C6
:1067F400ADFA15B0F0BDC04600240140341002408B
:08680400440F002008000240CF
:10680C0080B50B480121016200211022072383600F
:10681C00C26001614161816106490160FF21023161
:10682C008180FDF7D3FA002801D002F0CBF980BDAE
:08683C00B411002000300240FD
:1068440081B000680849884201D001B07047012036
:10685400000306490A6802430A600968014000917E
:10686400009801B07047C046003002403810024022
:1068740010B58AB01348144901600024099408949F
:106884000794069404F094FC002801D002F09EF9C9
:10689400059404940394029401940A4801A922469D
:1068A400FDF700FB002801D002F090F9054801A98A
:1068B4001022FDF7F7FA002801D002F087F90AB098
:0C68C40010BDC046F4110020007400401C
:1068D00070B586B000240594049400681549884278
:1068E00001D006B070BD01204107134A93680B43E5
:1068F000936093680B400093009911680143116005
:106900001168014000910394032502953020019005
:1069100000980520000701A9FDF732FE1126304638
:1069200029462246FDF7F4F93046FDF711FA06B084
:0C69300070BDC0460074004034100240EE
:10693C00F0B581B01649086801221043086015486B
:10694C00002380244025144E03273F030762066072
:10695C004360D602570291038160C56004614761B0
:10696C008661C3610A490968114000910099FDF7DD
:10697C0021FB002801D002F025F909240121002275
:10698C002046FDF7BFF92046FDF7DCF901B0F0BD5C
:0C699C0038100240E80E00201C000240F1
:0869A80000487047EE070000F3
:1069B000F0B585B0FDF768FD002801D0012434E072
:1069C000012046021A4D2968B1432960022401942E
:1069D0000490184800680006400E801E039001A82D
:1069E0006946FDF771FD00281AD13720C443124FC4
:1069F000124DE1192819826BC36B0120FDF7CAFC07
:106A000000280BD10834F4D10949086830430860E4
:106A1000FDF74EFD411E8841840006E00324044D2D
:106A2000286830432860FDF743FD204605B0F0BDDF
:106A300000200240E075FF1F38F00108C00500206B
:106A4000F0B583B03721CB4302461632264C274996
:106A50001D5DCE183827F5555B1CF9D30B681380E4
:106A60001B0C53808B8A02934B8A01938B89009372
:106A70004E890F89CC888B88CD8A958543830B8B73
:106A8000D38584834B8B1386C7838B8B5386CB8BA9
:106A90009386CB89D3860B8A13870685009B438711
:106AA000019B8387029BC3870B8C114C2380002B97
:106AB00001D0012353870A6B0281120C4281888D19
:106AC000382805D1C88D002805D0032003B0F0BDBB
:106AD000022003B0F0BD2420085C6538411E8841C7
:106AE000800003B0F0BDC04638F00108C0050020AA
:046AF0004A0D00202B
:106AF400B0B5C38A048B058D1B4A5581458B95809F
:106B0400858BD580C58B1581458F9581858F558261
:106B1400C58F95822404E3181360034616339C8DB5
:106B2400D482DC8D14831C8E54835C8E94839C8E5F
:106B3400D4835624045B1484DC8ED4811B8F2424D8
:106B44006525155513823823D362936A5B1C9362BF
:106B5400002904D001894089000440181063FFF71C
:0C6B640025FF411E8841B0BDC005002087
:106B7000B0B50B490B48024638C938C238C938C2CB
:106B800038C938C22421652242543821C162816A41
:106B9000491C8162FFF70CFF411E88414000B0BDD7
:086BA00000A90008C005002057
:106BA800024800786538411E8841704724F0010882
:106BB800F0B585B0FDF764FC002801D0012434E06D
:106BC800012046021A4D2968B14329600224019424
:106BD8000490184800680006400E401E039001A863
:106BE8006946FDF76DFC00281AD11720C443124FDF
:106BF800124DE11928198269C3690120FDF7C6FB06
:106C080000280BD10834F4D10949086830430860DA
:106C1800FDF74AFC411E8841840006E00324044D28
:106C2800286830432860FDF73FFC204605B0F0BDDA
:106C380000200240E075FF1F18F80108E804002052
:106C480080B5064800210182016041608160C16011
:106C5800FFF7AEFF411E8841400080BDE8040020D8
:106C680030B50121090240181721CA430D4B0E49BE
:106C7800D45C8D182C76521CFAD30A8802804A8874
:106C880042808A888280CA8802820A89C2804A89A8
:106C980002818A894281CA898281098AC181002048
:0C6CA80030BDC04618F80108E8040020C8
:106CB40080B501210902425A41180C4802804A88D1
:106CC40042808A8882800A8AC280CA8802810A89AC
:106CD40042814A8982818A89C281C9890182FFF7F6
:106CE40069FF411E8841400080BDC046E804002081
:106CF400F0B589B0002408944A480168042211437D
:106D04000160016811400391039901682022114335
:106D14000160016811400391039901680125294329
:106D240001600168294003910399016802273943EE
:106D340001600168394002970391039901680822B0
:106D44001143016000681040039003986903364EB4
:106D540030462A4604F040FAA9033046224604F09D
:106D64003BFA32481F210091224604F035FA30489C
:106D74003946224604F030FA079406940595032018
:106D84004003049004AF30463946FDF7F7FB069400
:106D94000594E8030190049030463946FDF7EEFB74
:106DA40007940694059500980490204E3046394681
:106DB400FDF7E4FB06950594FF200002049030469D
:106DC4003946FDF7DBFB0694059409200002049084
:106DD4000520060730463946FDF7D0FB0695059495
:106DE400C020049010483946FDF7C8FB0695059469
:106DF4000198049030463946FDF7C0FB0794069489
:106E04000595029804900A4E30463946FDF7B6FBC4
:106E1400069505940C20049030463946FDF7AEFBE8
:106E240009B0F0BD341002400008005000040050C6
:046E3400000C0050FE
:106E380070B50D46064600240A49204603F036FD83
:106E48002046314603F032FD0749204603F02EFD67
:106E58002046294603F02AFD0449204603F026FD72
:106E680070BDC04671BB000875A9000863B600086C
:106E780070B50D46064600240A49204603F016FD63
:106E88002046314603F012FD0749204603F00EFD67
:106E98002046294603F00AFD0449204603F006FD72
:106EA80070BDC04679BB000875A9000863B6000824
:106EB80070B50D46064600240A49204603F0F6FC44
:106EC8002046314603F0F2FC0749204603F0EEFC69
:106ED8002046294603F0EAFC0449204603F0E6FC74
:106EE80070BDC04681BB000875A9000863B60008DC
:106EF80000B585B0D84801260660FCF75DF900F0BA
:106F080065FCFFF7F3FEFFF715FDFFF793FB03F0B2
:106F18007DFAFFF777FCFFF7A9FC03F0C1F903F04E
:106F2800A3F903F053F903F02BF903F003F903F085
:106F3800D1F803F065F9C94C20460830872149008B
:106F480003F0C8FB0020C64921606060C548FEF711
:106F58004FF9002803D0C448C449FFF7A9FF00200F
:106F6800C34904F01BFAC048C249FFF761FFC24D8C
:106F78002868C2490140C248081811280FD8C149D9
:106F88007844007940008744080A0A0A0A0A0A0A6B
:106F98000A0A0C0A0A0A0A0A0E0FBB4904E0BB498E
:106FA80002E0BB4900E0BB49AF4C2046FFF740FF79
:106FB8002868030C0027B8493846224604F0EEF941
:106FC80003F02CFF0246B549384604F0E7F9FFF70D
:106FD800E7FC0246B249384604F0E0F9B149962286
:106FE800384604F0DBF9FDF727FF0246AE4938467C
:106FF80004F0D4F9FDF720FFAC4988420AD89A4C2E
:10700800AB492046FFF754FFAA492046FFF750FF37
:10701800FCF7B6FE00F01AFC00F04AFCFFF7C0FDD2
:10702800002807D09048A449FFF722FFFFF79CFDEE
:10703800FFF706FE8948FFF7FFFC002803D08A48BF
:107048009E49FFF735FF854C2046FFF709FE0028CB
:1070580003D085489A49FFF72BFF3002215A491C73
:107068002152E18F6E204843642103F0ABFA40219E
:107078006052944806604620205A4A21615A41438A
:1070880091480160E08B914902252A4603F0C9FE28
:10709800E08A218B628B8E4B01938E4B00936F2A73
:1070A80000D02E46652A00D03746090409188A4DB3
:1070B8008A4B28463A4603F00AFF894804F012F83A
:1070C800002801D0874906E08548FCF7CFFD002855
:1070D80000D1FCE284496448FFF7EAFE83480026B1
:1070E800314603F009FD07461021804803F004FDEE
:1070F80003907F495C4A30463B4604F04FF97D498E
:1071080004963046584A039B04F048F9012003903E
:1071180000F006FC724878490622FCF7AFFA00280E
:1071280003D051487549FFF7C3FE7548016804222A
:10713800914301606D48049E314603F09FFC10277F
:107148006A48394603F09AFC684831463246334665
:1071580003F0BDFC654839463246334603F0B7FCB8
:1071680000F05AFC67496848086068486849016047
:1071780068480160684801606848016068480160C3
:107188006848694904E00398684908706348684991
:10719800016008E00020208400F05CFFFCF754F850
:1071A800B04200D001E100F0CFFE284604F004F917
:1071B800002810D0284602F0C9FC022807D15D48F3
:1071C8000068002807D0284602F010FD03E0882058
:1071D8002221424A11505427E05B57490988401A36
:1071E8004142414152202152394801801A480068E1
:1071F8000028CFD02621208C0028CDD0695C00291A
:10720800CAD14E49884200DDA6E0411E1D2900D999
:10721800EEE149007944898849008F4494002301AC
:107228003401ED015301ED01ED01ED01ED016A01BC
:10723800ED01ED01ED01ED01ED01ED01ED01ED01D6
:10724800ED016D01ED01ED01ED01ED01ED01ED0146
:10725800ED01ED01ED019100A4120020340C002095
:10726800CA0001003810002023B9000828B9000816
:107278003DB9000842B9000800580140FF0F00005E
:10728800AAFBFFFF65B60008A9B6000889A900088F
:1072980087B60008CBB6000889BB0008EDB6000821
:1072A800A5BB000823B7000853B90008FF8FD00317
:1072B800D9BB0008DCB30008F1BB000864B90008BA
:1072C800EFB30008701200201C04002000040050D6
:1072D800661300205C040020F8090020F40D00204B
:1072E800840E0020B2B900081EB40008F411002072
:1072F800C3B90008F0B900088213002045B7000898
:1073080008000240F4120020997E0008F0120020C4
:10731800F9010020EC1200202C1300201C1300207F
:107328003C130020F8120020E97E000864130020B6
:10733800158A0008240400204A0D00204F4F000041
:1073480002F0DCF826E700212046FFF7CFFB0028F3
:1073580000D1F7E0E449F2E0FB4988420FDCE34959
:10736800884200D1CCE0FC49884200D1CCE0FB49FE
:10737800884200D040E1F148F14901600AE7F34949
:10738800884200D1CAE0F249884200D1D0E0F149F0
:10739800884200D030E1E8480068E349884200D0DC
:1073A800F8E6E548EE490160F4E60746E248006879
:1073B8008047DC4800688047D94800688047DB4838
:1073C80000688047DA4800688047DA4800688047E4
:1073D800EE4E306840003060052000070121890327
:1073E80003F093FB31680143316002D0384600F066
:1073F8006BFE384600F0F6FF384601F097FA04981D
:10740800381AE34988420ED3BA48E249FFF710FD1B
:10741800BB4800680028049705D02046FFF746FCC3
:107428000020B7490860A08D022800D195E0012806
:107438003E4600D0B7E6D8480068012800D0F3E0FF
:1074480009263046FCF78CFCEA2000212152D84856
:10745800D84901603046FCF777FCB648D649016048
:107468003E46A0E6608B6F2800D1A9E0652800D0D1
:10747800B0E0E08A218BA44A0092A24A0192090452
:1074880009180022AFE0FFF76FFB0028994F03D0DF
:107498003846B949FFF70CFDFFF7D2FB2046FFF746
:1074A800CBFA002803D038469349FFF701FD204660
:1074B800FFF7D6FB002800D16CE68E488F49FFF70E
:1074C800F7FC67E68B48AD49FFF7B2FCE15B9D48E6
:1074D8000088814208D100212046FFF707FB56208B
:1074E800205AE05397490880411E88415021605234
:1074F80050E602F049F84DE6002000F011FA49E69E
:1075080089488E49086045E68B4800688649884264
:1075180000D03FE68848934901603BE6864800680A
:107528008149884200D035E683488F49016031E6B9
:1075380001212046FFF7DAFA002803D08D496D486B
:10754800FFF7B6FC2046FFF777FA002800D121E6BE
:1075580068486949FFF7ACFC1CE698480068411E7A
:10756800484248418C4909680129039900D00146DD
:10757800012967D19248007800283E4600D012E6DB
:1075880009263046FCF7ECFBEA2000212152884806
:10759800884901603046FCF7D7FB7F48006801281E
:1075A80002D164488449016084480068012802D1F6
:1075B8006048854901600398814908703E46F2E5B4
:1075C800E08A218B504A00924E4A01920904091818
:1075D800012208E0E08A218B4B4A0092494A019235
:1075E8000904091802222846484B03F070FCD1E52B
:1075F8007D21890088425AD0614802680121C94327
:10760800116100275762FDF729FE0028394904D087
:1076180008465C49FFF74CFC364935480760084680
:107628005949FFF725FCB5E55C480068012800D1F9
:10763800ACE55B480068012830D05A48006801284A
:1076480032D0B0E555480068012806D15C4800787A
:1076580000283E4600D0A6E595E551480068012877
:1076680005D15748007800283E4614D09BE54D4880
:107678000068012805D15248007800283E4610D0FD
:1076880091E54F4E31784F480268384690470020C0
:1076980030703E4687E503984949087025484349B4
:1076A80076E503984649087022483F4970E51B482B
:1076B8000068002181604161EA202152BFF34F8FA9
:1076C8002A482B490160BFF34F8F00BFFDE71048E0
:1076D80003F066FD3F210143009100200D490E4A49
:1076E800044B03F05BFEF9E4F3B80008504F0000C8
:1076F800A412002023B9000864B90008EFB30008F9
:1077080070120020661300205C040020F40D002095
:10771800840E002091B900081DBC0008F411002057
:10772800F4120020F0120020F9010020EC120020D1
:107738002C1300201C1300203C130020F8120020FA
:10774800E97E00084A0D00206D9D00006E9D000036
:10775800E3C4000058EC0000F9750000C57600008D
:1077680005960008899600087D9700080CED00E052
:107778000400FA0579BD000830B6000819B60008FB
:10778800841000209DBD000833BB000810040020B1
:10779800C1D401001DBA00086C1200208412002018
:1077A8008812002080120020E98A00087D8A0008DB
:1077B800DC12002001000020B1890008901200208E
:0C77C800641300204C1300205D8B0008AF
:1077D40070B592B00025069501267002FDF72AF8CF
:1077E400700711907006109070040F9010200E9086
:1077F4000D9502240B940A964020099030020790BC
:10780400300405900B20049003200C90C0020890D3
:1078140004A8FDF739F8002803D00B480B49FFF7FB
:1078240049FB039502950720009001946846214680
:10783400FDF74AFA002803D003480449FFF73AFB4E
:10784400FDF754FB12B070BD23B900080EB6000852
:10785400F0B581B0164C0125204629462A4603F08E
:10786400BBFC0221009120462A4603F0B5FC042704
:10787400204639462A4603F0AFFC7D26F000FBF78C
:10788400EBFC00240A482946224603F0A5FC084DD7
:1078940028460099224603F09FFC28463946224692
:1078A40003F09AFCB000FBF7D7FC01B0F0BDC04672
:0478B400000400507C
:1078B800B0B5134D29681348134C30232246FCF702
:1078C800F1FB002804D011481149FFF7F1FAFEE74F
:1078D8000E481049FFF7ACFA7D20C2000948002184
:1078E800FCF7C6FC002804D008480B49FFF7E0FA6B
:1078F800FEE706480949FFF79BFA2C60B0BDC04671
:1079080008ED00E0E80E00200005002023B900087B
:1079180063B7000835B40008A1B7000825BC000803
:10792800F0B581B00546FBF78FFC0446284A0126CE
:107938003702002D07D11068201A3946F4318842E1
:1079480001D801B0F0BD15462248FDF7BFFC224919
:10795800888D002800D02C6000258D8509242046BC
:10796800FCF7FEF9EA201C490D521C481C4901602D
:107978002046FCF7E9F9F1431A48026811611A49EF
:107988001A4B0B601A491B4B0B601B491B4B0B60B6
:107998005562FDF763FC1A480068076071020160D0
:1079A8003003184908600C20FCF7CEF94520800008
:1079B80009490D52892040000D52134805601348AB
:1079C8000560134805601348056001B0F0BDC04666
:1079D80094120020D0100020340C0020DC1200206B
:1079E80001000020681100201C130020958C00085D
:1079F8002C130020118D0008F01200209D8D000826
:107A0800840E002080E200E0841200206C12002026
:087A18008812002080120020FA
:107A2000F0B583B001252E02F54C2046314603F017
:107A300070F802956D02012825D12046294603F0F1
:107A400068F801281FD10127B902204603F061F828
:107A5000012818D13D46F902204603F05AF80028C3
:107A600000D1FEE0E748E549FFF7E6F9E748F549C8
:107A7000FC4AFD4BEA4FFD4E3E6003604260816070
:107A8000C160002070E12046314603F042F8002832
:107A900025D12046294603F03CF801281FD10127B3
:107AA000B902204603F035F8012818D1F902204622
:107AB00003F02FF8002800D1FCE0D248EF49FFF78F
:107AC000BBF9D248DF49E04AE04BD54DE04E2E608D
:107AD0003D46036042608160C160384644E1204613
:107AE000314603F016F8012824D12046294603F038
:107AF00010F800281ED10127B902204603F009F82A
:107B0000012817D1F902204603F003F8002800D11C
:107B1000E2E0BC48D249FFF78FF9BC48C949D14AD5
:107B2000D14BBF4DD14E2E60036042608160C16079
:107B3000022018E12046314602F0EBFF002824D154
:107B40002046294602F0E5FF00281ED10127B90290
:107B5000204602F0DEFF012817D1F902204602F08C
:107B6000D8FF002800D1DCE0A648B549FFF764F94A
:107B7000A648B449B44AB54BA94DB54E2E60036032
:107B800042608160C1600320EDE02046314602F092
:107B9000C0FF0299CF0201280CD12046294602F0ED
:107BA000B8FF012806D101908102204602F0B1FF02
:107BB00000283DD02046314602F0ABFF00280BD113
:107BC0002046294602F0A5FF012805D18102204662
:107BD00002F09FFF002855D02046394602F099FF59
:107BE000002811D087488849FFF726F98748884937
:107BF000884A894B894D056043608260C16088482E
:107C000088490160042010E07E488749FFF714F995
:107C10007E487F497F4A804B804D0560436082608B
:107C2000C1607F48814901600C2002990D469CE0AB
:107C3000019E2046394602F06CFF00285DD0714855
:107C40007D49FFF7F9F871487149724A724B734DDB
:107C5000056043608260C160714872490160042020
:107C60005CE068488749FFF7E7F868487549814A4A
:107C70007D4B6B4F804E3E60036042608160C1600F
:107C8000082071E02046394602F043FF002859D011
:107C90005C486749FFF7D0F85C485D495D4A5E4B38
:107CA0005E4D056043608260C1605D485D49016072
:107CB000052058E053487249FFF7BEF85348614920
:107CC000654A624B564D654E2E600360426081608E
:107CD000C1600920012547E04A486549FFF7ACF833
:107CE0004A485849634A604B4D4D634E2E600360CD
:107CF00042608160C1600A2035E042484F49FFF789
:107D00009BF842484249434A434B444D0560436017
:107D10008260C1604248454901600C2002993546A5
:107D200023E038484B49FFF787F8384845494A4A25
:107D3000464B3B4D494E2E60036042608160C160FE
:107D40000B2010E02F483B49FFF776F82F483049C9
:107D5000304A314B314D056043608260C16030482C
:107D6000324901600D2000250299474F7885474828
:107D700005700903204602F0CCFE002803D04448D9
:107D80000021016006E0424801210160788D102148
:107D900001437985012675032046294602F0B9FE84
:107DA000002803D03B480021016005E03948066007
:107DB000788D20210143798531022046FCF7B6FCFD
:107DC00071022046FCF7B2FCB1022046FCF7AEFC83
:107DD000F1022046FCF7AAFC31032046FCF7A6FC82
:107DE00020462946FCF7A2FCB1032046FCF79EFC86
:107DF000F1032046FCF79AFC03B0F0BD68B400081C
:107E00000004005023B9000852BA000828120020CC
:107E1000D193000855930008DD9200087192000884
:107E20004C1300203994000855BC0008D591000877
:107E30003FB50008A9B8000814B500087FB80008CD
:107E4000E9B40008F9010020719100085990000878
:107E5000ED90000855B800089D900008D98F0008E3
:107E6000BEB40008758F00085D8E0008F18E000812
:107E70002BB80008A18E0008DD8D000893B400081F
:107E800001B80008D7B70008340C0020FB0100201F
:087E90008C120020B412002046
:107E9800F0B581B0FBF7D8F904460D4F3868201AC1
:107EA8000C490E78002E03D033280ED3002203E0AD
:107EB8000949884209D9012208480125294603F0C1
:107EC80089F93C606E400348067001B0F0BDC046B9
:107ED800441300207C130020B60300000004005067
:107EE80080B511480068002181604161EA220F488D
:107EF80081520F490F4A0A600F490968002900D0CA
:107F080080BD0E490A68002A07D111221201835A3E
:107F18005B1C83520A480122026001200860FBF7BB
:107F280093F90849086080BDF4110020340C002042
:107F3800DC120020F90100208412002080120020A9
:087F4800701200201404002057
:107F5000F0B581B0FBF77CF9324908600A68324815
:107F60000368D21A022A2ED3096801602F4D688F48
:107F70002F4909684018E821685201B24B2080005F
:107F800048432C4902F002FBD8216B5E2A4A146850
:107F9000E31AC318963BD817800C18188013685240
:107FA0001360EA26AB5B002B0AD0244C2778002F05
:107FB0000BD0022B10D100042749884212DD02E0C9
:107FC0001E480021017001B0F0BD00206852106011
:107FD0000120207001B0F0BD032BF4D10004194939
:107FE0008842F0DB164F38680028ECD1092420467F
:107FF000FBF7BAFE14480068002181604161A95373
:108000001248134901602046FBF7A2FE872040007A
:10801000295A491C2952012038600E49086001B0D4
:10802000F0BDC0465C13002060130020340C00201B
:1080300074120020FF0F000058130020801300204E
:108040008812002001003C00F4110020DC12002006
:0C805000F901002070120020FFFFC3FFA8
:10805C0080B5FBF7F7F816490A68904200D180BD4D
:10806C00086001F0D9FF082002F014F8002806D0AF
:10807C0010481149FEF7DAFE01F03EFA80BD0820E7
:10808C0002F016F8002806D00A480C49FEF7CEFE7E
:10809C0001F078FA80BD042001F0FCFF0028DED04E
:1080AC0004480749FEF7C2FE0020FFF737FC80BDED
:1080BC00E812002023B90008D3B800086AB50008FC
:0480CC00A1BC00084B
:1080D000F0B581B0A0490A68821A4E2A00D238E170
:1080E000086000259D499E4C9E4B2846224603F081
:1080F00059F99D4F9D4A28463946234603F052F9C7
:10810000D8209B4E325E9B49284603F04BF9284607
:108110003946964A234603F045F9FC20325E9649DB
:10812000284603F03FF928463946904A234603F093
:1081300039F9EC20325E9149284603F033F928469C
:1081400039468A4A234603F02DF9CC20325A8C490D
:10815000284603F027F928463946844A234603F087
:1081600021F9D220325A8749284603F01BF92846C4
:1081700039467E4A234603F015F9CA20305A824E0A
:10818000824C0028324600D022468149284603F01E
:1081900009F928467449754A714B03F003F9C82060
:1081A0007349085A002800D026467A4928463246A4
:1081B00003F0F8F828466C4F39466C4E3246684B4F
:1081C0001C4603F0EFF874480068C26A73492846F9
:1081D00003F0E8F8284639463246234603F0E2F831
:1081E0006D480068026B6E49284603F0DBF82846AC
:1081F00039463246234603F0D5F8EA205C49085A4E
:10820000002803D0012803D1674A06E0654A04E04C
:10821000022801D0664A00E0644A002465492046ED
:1082200003F0C0F8504D514A4D4F204629463B4679
:1082300003F0B8F8E2204E4E305E5F494143CA0F6A
:1082400089148A180921C94351430818C1174840A5
:10825000431A5A49204603F0A5F820462946434AC6
:108260003B4603F09FF8F625705BC00704D0002062
:108270005349544A03F096F85149534A204603F0B3
:1082800091F83949394A364B204603F08BF8705B38
:10829000800704D500204A494A4A03F083F8484938
:1082A0004A4A204603F07EF82F49304A2C4B20469C
:1082B00003F078F8705B400704D500204049414A3C
:1082C00003F070F83E49424A204603F06BF8264915
:1082D000264A234B204603F065F8705B000704D55F
:1082E00000203749374A03F05DF83549394A2046BE
:1082F00003F058F81C491D4A194B204603F052F868
:10830000705B800604D500202D492E4A03F04AF800
:108310002B49274A204603F045F81349134A104BCE
:10832000204603F03FF82C48022102F0F2FB01281E
:1083300006D1002022492A4A03F034F8294A00E0F5
:10834000264A1F49204603F02DF82749204603F00E
:1083500029F801B0F0BDC046381300209FBA0008CC
:108360001DBC000823B90008C1BC0008B9BC000846
:10837000340C0020C9BC0008D5BC0008A4BA000811
:1083800085B5000890B50008E9B80008E1BC000810
:10839000ADBA0008B6BA0008F41100209BB5000879
:1083A000A6B50008B1B50008B4B50008B7B5000817
:1083B000BAB50008EBB8000867660000BFBA00084D
:1083C000BDB50008F1BC0008C0B50008C3B5000881
:1083D000C6B50008C9B50008000C005009BD00086A
:0C83E000F9BC000801BD0008F1B800085D
:1083EC00F0B589B0BD4909780029BD4D01D12946A8
:1083FC0000E08721BB4C2268821A8A4200D81EE218
:10840C00CC26B94B995BB94A1268571AF9178F43A6
:10841C00B749CA886A43110B0A2251437918CF080D
:10842C009F5301260296AD4D2E702060AF4801601F
:10843C00B8B21E46D021595A814203D2D033A84D2E
:10844C00AB4F06E0CE21715A8142A54DA84F01D900
:10845C00CE331880D220315AA64B1C68611ACC1727
:10846C00A1437C886C43240B624389184A0932521D
:10847C00196090B2FC49884212D8FC4A1168002954
:10848C0019D1F621735A08241C43745283214900D4
:10849C00735A5B1C7352029B1360FA490B600AE01F
:1084AC00F649884207D3F621725A08239A4372522E
:1084BC00F34900220A60D621715A814202D2324617
:1084CC00D63205E0D421715A814202D93246D432D7
:1084DC0010803888EC494143EC480818EC4902F00C
:1084EC004FF8E221725EEB4B1C68A21A1018EA4A94
:1084FC008218D017C00E1018401170521A6004B2B6
:10850C00E621715E8C4202DD3146E63105E0E42164
:10851C00715E8C4202DA3146E4310880318D8C4236
:10852C0013DA4B204843642102F04AF8A0421DDDC7
:10853C00DB480068002819D0F620315A029A914382
:10854C003152D6480021016010E0D448016800295E
:10855C000CD1F621725A029B1A43725281214900A6
:10856C00725A521C72520360C6480360CD480068B0
:10857C00401E414241414900F620325A26239A437B
:10858C005118C94A1268521E534253419A0051184D
:10859C00C64A1268521E534253415A01891831522D
:1085AC00D823F05E0028009305D4DC21725A904247
:1085BC000ADCDA2105E0E021725A4042904203DCE9
:1085CC00DE21725A904200DA7052B9490868F822DA
:1085DC00B052B8480268FA23F252B74A1268B74B45
:1085EC001B689A1A09688D18E917090F69180A117E
:1085FC004C21715A9142019201DC561A00E000267E
:10860C00AF490968AF4A1268511A00684718F81741
:10861C00000F381804114E209649085A001B00DC34
:10862C00361893487043A84901F0AAFFFC21914ADF
:10863C005052A2480560A348076017469E4801990E
:10864C0001609F4804605F2084006643D18F3046F0
:10865C0001F096FFEC217852EA257A5B9B48016881
:10866C00002A019404D19A4B994201D0984A09E00E
:10867C00012A04D1974A914201D0964A02E0964AC7
:10868C00914200D00260954C4021204602F03BFA0A
:10869C0006468021204602F036FA914909784A4272
:1086AC004A41B11A4B1E9941CA23F952801A411EF4
:1086BC008841C8217852785B401E02281CD800984B
:1086CC00385E032800DABCE086480221012202F061
:1086DC007FFD019978318448016012E0701300200D
:1086EC00B80B000010130020340C002040130020A5
:1086FC0082130020400400207A480221002202F05C
:10870C0067FD029E44203D5A784C2188A94214D022
:10871C00B98F8D4211D956494A1E954201D9395209
:10872C000D466948684301F04BFF4621785225807D
:10873C004A21795A41436E48016048203D5A6D4C9C
:10874C002188A94210D01E2D01D81F253D526A4800
:10875C0068436A4901F034FF4A217852258046214A
:10876C00795A41436248016005200007310202F04A
:10877C00CAF9401E41424141FE2039524225785BE4
:10878C0000265F4CA15F814259D05E4802F02CF963
:10879C00785BBA8F9042014600D811469042344A19
:1087AC0001D3914204D9914200D311467953084622
:1087BC0020800196089644494843114601F000FF79
:1087CC000790514805900320860504964F48039066
:1087DC00029806904B4803A9FBF7D0F8002803D069
:1087EC004B484C49FEF762FB03AC029820734A4895
:1087FC00059004964948039001980890795B32489B
:10880C0048431B4901F0DCFE07903E482146FBF72C
:10881C00B5F8002803D03E483E49FEF747FB3948DF
:10882C0015490622FAF728FF002803D038483C499E
:10883C00FEF73CFB3B48016804229143016009B000
:10884C00F0BD0028029E00DD5CE72749086801287E
:10885C0001DB401E0860002800D053E721480221AC
:10886C00002202F0B5FC4DE71F4E000090120020D4
:10887C00B80B0000340C002082130020C15D0000F6
:10888C009012002070120020140500000CE3F7FF7A
:10889C00EF06000004130020D4FEFFFF6C12002032
:1088AC00B4120020841200208012002088120020B4
:1088BC00781200207C120020FC12002008130020EB
:1088CC00001300200C130020FF0F0000F0120020FA
:1088DC009D8D0008BD8D0008518D000800080050CA
:1088EC00FB010020000C0050141300206E1300201C
:1088FC001C0400207213002000E2040040420F0010
:10890C006A130020840E002004000008FFFF1700EB
:10891C0023B900080EB6000840000018FFFF27001E
:08892C0045B7000808000240F5
:10893400B0B517490A68821A1A2A0FD30860154D70
:10894400287840002870052000070124E10302F084
:10895400DEF82978002802D0002911D0B0BD2143C7
:1089640029700D4801780029F8D104700B4801687A
:10897400002908D00021016009480A490160B0BDFE
:1089840005480170B0BD0460054807490160B0BDE9
:10899400C8120020E70400206813002024040020EB
:0C89A400F4120020E58B0008997E00080A
:1089B000F0B587B005AD0F48288006AEC8203080DE
:1089C000082003900C4F0297019500960B480C4924
:1089D0000C4A0124234602F045FA02200096019534
:1089E0000297039008480949094A234602F03AFAD7
:1089F00007B0F0BDC4090000000400502813002097
:108A00002413002020130020C4120020C0120020D4
:048A1000BC12002074
:108A1400F0B587B005ADC820288006AE30807080E0
:108A24000D486880082003900C4F0297019500962A
:108A34000B480C490C4A0224234602F011FA009612
:108A4400019502970394094809490A4A234602F00A
:108A540007FA07B0F0BDC046C40900000004005086
:108A6400281300202413002020130020C412002007
:088A7400C0120020BC1200201A
:108A7C00F0B589B005ADC820288007AE3080708075
:108A8C006880B0800D48A880082003900C4F029796
:108A9C00019500960B480C490C4A0324234602F01E
:108AAC00DBF90220009601950297039008480949CA
:108ABC00094A234602F0D0F909B0F0BDC409000000
:108ACC000004005028130020241300202013002041
:0C8ADC00C4120020C0120020BC120020B8
:108AE800F0B589B0002005AAC821115207AA115271
:108AF800801C0628F7D105AD0E48E88007AEF18046
:108B0800082003900C4F0297019500960B480C49DA
:108B18000C4A0424234602F0A1F90220009601958C
:108B28000297039008480949094A234602F096F932
:108B380009B0F0BDC409000000040050281300204B
:108B48002413002020130020C4120020C01200208B
:048B5800BC1200202B
:108B5C00F0B58BB0002005AAC821115208AA1152F9
:108B6C00801C0828F7D105AD0E48288108AE31814C
:108B7C00082003900C4F0297019500960B480C4966
:108B8C000C4A0524234602F067F902200096019551
:108B9C000297039008480949094A234602F05CF9F8
:108BAC000BB0F0BDC40900000004005028130020D5
:108BBC002413002020130020C4120020C012002017
:048BCC00BC120020B7
:108BD00080B502480249FEF76FF980BD23B900084D
:048BE0000EB60008C5
:108BE40080B5044801210A4602F0F6FA0248034916
:108BF400016080BD00040050F4120020F90100203F
:108C04000348006800218160416102480180704787
:088C1400F41100201E0D0020E8
:108C1C00F0B589B005ADC820288007AE30807080D3
:108C2C001148E8807D2080006880A880C830B08022
:108C3C00F080082003900D4F0297019500960C4888
:108C4C000C490D4A0424234602F006F90220009632
:108C5C00019502970390094809490A4A234602F0F4
:108C6C00FBF809B0F0BDC046C40900000004005078
:108C7C00281300202413002020130020C4120020ED
:088C8C00C0120020BC12002000
:108C9400B0B5084C0821002520462A4602F09CFA6B
:108CA400022120462A4602F097FA0348034901604C
:108CB400B0BDC046000400501C130020F901002080
:108CC400F0B581B0FAF7C2FA04460D4E3068201AA6
:108CD4000C4D2F78002F03D0C9280ED3002204E0B6
:108CE40019214901884208D901220748102102F0BC
:108CF40073FA3460012047402F7001B0F0BDC046C4
:0C8D040030130020781300200004005001
:108D100080B504481021002202F060FA024803499D
:108D2000016080BD000400502C130020F9010020D8
:108D300080B504481021012202F050FA024803498C
:108D4000016080BD000400502C130020F9010020B8
:108D5000F0B581B0FAF77CFA04460C4E3068201A60
:108D60000B4D2F78002F03D033280DD3002203E0C2
:108D70000849884208D901220748042102F02EFA46
:108D80003460012047402F7001B0F0BD181300205F
:0C8D900074130020B60300000004005023
:108D9C0080B504480421002202F01AFA0248034963
:108DAC00016080BD00040050F0120020F901002089
:108DBC0080B504480421012202F00AFA0248034952
:108DCC00016080BD00040050F0120020F901002069
:108DDC00B0B5002901D0022523E013490A68821A94
:108DEC00124C23689A421ED908601148802101F068
:108DFC008AFE454245410F490978002900D00546B5
:108E0C000D480068A84202D10C490D4803E0A800A7
:108E1C000C4908580C49AA000C4B985089582160F1
:108E2C00804705480560B0BD54130020580400204D
:108E3C0000080050FB010020540400202CA900085D
:108E4C00F90100202812002024A90008601200203B
:108E5C0010B509242046FAF781FF084801F062FB9F
:108E6C000B48012101800648064901602046FAF7AB
:108E7C0069FF05480549016010BDC046650000202A
:108E8C00DC120020310300202C130020C58C0008BC
:048E9C001E0D002087
:108EA000B0B509242046FAF75FFFEA200A4D0021F9
:108EB00029520A480A4901602046FAF749FF212051
:108EC000C000295A491C2952064807490160074831
:108ED00001210160B0BDC046340C0020DC1200202E
:108EE000890000202C130020C58C0008701200207F
:108EF000B0B5002902D00020C54323E013490A6819
:108F0000821A134C23689A421ED9086011488021A6
:108F100001F0FFFD454245410F490978002900D085
:108F200005460E480068A84204DAA8000E49085811
:108F30000E4901E00A490B48AA000D4B9850895888
:108F40002160804705480560B0BDC046E41200209E
:108F50003C04002000080050FB01002038040020E1
:108F60002CA90008F90100202812002024A90008DB
:048F7000501200207B
:108F740070B509242046FAF7F5FEEA200E4D0026C6
:108F84002E520E480E4901602046FAF7DFFEAE85E8
:108F94000124E1430B48026811610B490B4B0B6040
:108FA4005662FCF75DF92120C000295A491C295258
:108FB4000748046070BDC046340C0020DC12002059
:108FC40001000020681100202C130020118D0008DE
:048FD40070120020F7
:108FD800B0B5002901D0022523E013490A68821A96
:108FE800124C23689A421ED908601148402101F0AA
:108FF8008CFD454245410F490978002900D00546B6
:109008000D480068A84202D10C490D4803E0A800A9
:109018000C4908580C49AA000C4B985089582160F3
:10902800804705480560B0BD48130020480400206B
:1090380000080050FB010020440400202CA900086F
:10904800F90100202812002024A900085812002045
:1090580010B509242046FAF783FE084801F064FA9F
:109068000B48012101800648064901602046FAF7AD
:109078006BFE05480549016010BDC046210000206F
:10908800DC120020310300202C130020C58C0008BE
:049098001E0D002089
:10909C00B0B509242046FAF761FEEA200A4D0021FA
:1090AC0029520A480A4901602046FAF74BFE8520EE
:1090BC004000295A491C29520648074901600748B3
:1090CC0001210160B0BDC046340C0020DC12002030
:1090DC00450000202C130020C58C000870120020C5
:1090EC00B0B5002902D00020C54323E013490A681B
:1090FC00821A134C23689A421ED9086011484021E9
:10910C0001F001FD454245410F490978002900D085
:10911C0005460E480068A84204DAA8000E49085813
:10912C000E4901E00A490B48AA000D4B985089588A
:10913C002160804705480560B0BDC046D8120020AC
:10914C002C04002000080050FB0100202804002003
:10915C002CA90008F90100202812002024A90008DD
:04916C004812002085
:1091700070B509242046FAF7F7FDEA200E4D0026C7
:109180002E520E480E4901602046FAF7E1FDAE85E9
:109190000124E1430B48026811610B490B4B0B6042
:1091A0005662FCF75FF885204000295A491C295275
:1091B0000748046070BDC046340C0020DC1200205B
:1091C00001000020681100202C130020118D0008E0
:0491D00070120020F9
:1091D40070B5002901D0042430E01A490A68821AC3
:1091E400194E33689A422BD90860184D40212846FD
:1091F40001F08DFC04468021284601F088FC4142A0
:109204004141134A1278002A00D00146604260416D
:10921400002A00D0204644000C430E4800688442D3
:1092240002D10D490D4803E0A0000D4908580D492D
:10923400A2000D4B9850895831608047054804605E
:1092440070BDC04650130020500400200008005098
:10925400FB0100204C04002044A90008F90100206F
:0C9264002812002034A900083812002055
:10927000B0B509242046FAF777FD0F4801F058F9F8
:109280000E480F4901602046FAF762FD124801219D
:1092900001800C480C4901600C4C08210025204637
:1092A0002A4601F09BFF022120462A4601F096FF44
:1092B000074808490160B0BDA9000020DC12002069
:1092C000310300202C130020C58C0008000400503E
:0C92D0001C130020F90100201E0D0020DE
:1092DC0070B509242046FAF741FDEA20114E03210E
:1092EC0031521148114901602046FAF72BFD104804
:1092FC0010490160104C0821002520462A4601F037
:10930C0067FF022120462A4601F062FF2120C0009F
:10931C00315A491C31520948094901600948012157
:10932C00016070BD340C0020DC120020CD00002048
:10933C002C130020C58C0008000400501C130020C6
:08934C00F9010020701200205D
:10935400F0B581B009252846FAF704FDEA20124F3A
:1093640002243C521148124901602846FAF7EEFCE7
:10937400104811490160114D082100262846324643
:1093840001F02AFF28462146324601F025FF8520B8
:109394004000395A491C395209480A4901600A48AF
:1093A4000121016001B0F0BD340C0020DC1200206A
:1093B400410100202C130020C58C0008000400503B
:0C93C4001C130020F90100207012002092
:1093D000B0B509242046FAF7C7FCEA200E4D00215B
:1093E00029520E480E4901602046FAF7B1FC2120AF
:1093F000C000295A491C295285204000295A491C7D
:10940000295208480849016008480949016009488B
:1094100001210160B0BDC046340C0020DC120020E8
:10942000B50100201C1300201D8C00082C13002007
:08943000118D000870120020EC
:1094380070B5002906D0264800210170C843254987
:10944800086070BD24490A68821A244E33689A421B
:109458003CD90860224D4021284601F056FB0446BD
:109468008021284601F051FB414241411D4A1278B2
:10947800002A00D0014660426041002A00D0204600
:1094880044000C43134D2868844207D1A100174AB1
:1094980018485050184A5158316015E00C48017866
:1094A800012903D1A000114908580BE0002C01D074
:1094B80001210170A1000C4840580C4A50500C4A38
:1094C80051583160002800D080472C6070BDC046DC
:1094D8006C13002030040020E01200203404002027
:1094E80000080050FB01002028120020181200205C
:0C94F80034A90008F901002044A9000874
:10950400F0B581B00220C643F9F7A0FE0446164D1B
:10951400A88DC01EB04224D8144E3068201A1449B5
:1095240088421ED313480068211A1348814218D96F
:1095340012490968611A814213D91148FBF7C8FE20
:109544000127F9430F480268116134600021516218
:10955400FBF786FE43208000295A491C29520A48F9
:10956400076001B0F0BDC046340C00209412002006
:10957400E903000014040020102700001804002050
:0C958400D0100020A00F0020701200206A
:10959000F0B581B00220C043154CA18DC91E814297
:1095A00021D81248006800281DD00125EE43F9F7A4
:1095B0004FFE10490A6816610F4B1860002757626A
:1095C0000846FBF74FFE0D4801680E614F62FBF73E
:1095D00049FE43208000215A491C21520848056059
:1095E0000C20FAF7C1FB01B0F0BDC0468C12002080
:1095F000340C0020EC0F002094120020D01000202A
:0496000070120020C4
:10960400F0B583B000252C462F4616480668164947
:109614000A680292036808680090002013492A46E9
:1096240001F0BEFE34190298C7196D1C104885421A
:10963400EBD105463846294600F0C6FF0646104FD2
:1096440078802046294600F0BFFF388082B2B3B24A
:109654000020084901F0A4FE07480849016003B04E
:10966400F0BDC046781200207C120020CCBA00085D
:1096740050C30000F9BA00083C130020F90100208F
:04968400800C002036
:10968800F0B581B02E482F49FDF7D2FBF9F7DCFD84
:109698000446F9F7D9FD001B2B4E0027B04215D21E
:1096A8003D46E81B294909680D18E817000F2818D6
:1096B8000711002026493A4601F070FE0120F9F70B
:1096C800C9FDF9F7C1FD001BB042EAD34E20214E77
:1096D800305A3C1AE220305EC72802DC6E20604314
:1096E80010E080B2C1084A2910D80A2141431A481B
:1096F800081880B2000919494143080C6E21081A5C
:1097080044432046642100F03DFF0446A5B26E2084
:109718006843642100F056FF40217052F4871048D6
:109728006043104900F02EFFB08783B200200E4935
:109738002A4601F033FE0D480D49016001B0F0BD25
:1097480023B90008CCB5000860EA00007C120020AC
:1097580011BD0008340C002030F8FFFF3E0A00005D
:10976800B80B0000FF0F000031BD00083C130020BB
:04977800F9010020D3
:10977C00F0B581B00024104F25463E683B680020B0
:10978C000E49224601F008FE7519641C0C488442EF
:10979C00F3D10146284600F013FF0A49081A0A497A
:1097AC00488702B20020094901F0F6FD0848094932
:1097BC00016001B0F0BDC04674120020F3B5000882
:1097CC0050C30000FF070000340C00201EBB000833
:0897DC003C130020F9010020FC
:1097E400F0B583B00D46029001600C203F4906C5D8
:1097F4000021E86029616961A961E96129620126A2
:109804003703083D2C4680340998089A002B04D06D
:10981400012B04D10321490202E0B10200E00F460A
:10982400AF602961511E4A1E91414903E96000F06D
:109834009DFE00272E4B3A4601F0ADFB00F07EFE64
:1098440001906068002803D12770284600F01AFEB2
:109854002420606028680168B14301602846FBF752
:10986400E1FE0128029C29D0A86A002802D02846DB
:1098740001F086F9B103286882680A438260F10323
:1098840082688A43826001681A4A0A400260F105CC
:1098940042680A434260B10602680A430260FF213B
:1098A400090642690A4001990A4342610168314349
:1098B40001602846FBF7BEFF002801D0FFF786F9B8
:1098C400206801F092FA002801D0FFF77FF92068A0
:1098D400273432022146FCF7B5F8002804D00648A4
:1098E4000649FDF7E7FAFEE703B0F0BD0038014092
:1098F40000000C40FFFF00FCBDBD000844BB000895
:10990400F0B58DB005460268D16910680C9001204D
:109914000A90000709900595843590680B90080714
:10992400089048D00998431C0B980340012637023D
:109934003C4620340C9804401C433CD007407C42F5
:109944007C41CF070A9F00D02746002F03D116621F
:10995400AC683443AC600B980640744274418F0782
:109964000A98074600D52746002F05D10224146221
:10997400AC6804272743AF60744274414E0706461F
:1099840000D52646002E05D104241462AC680226B4
:109994002643AE60089800280DD55C1EA3410C98A0
:1099A40084060A9C00D41C46012C04D108231362AB
:1099B400AC681C43AC600126F00507900B050FD57D
:1099C4000B9B0340B4060C980440E31808D0F30240
:1099D400136220236B602B605A4B1E755A4C1E5524
:1099E400049620200F460890074022D00B9B09982C
:1099F40003400C9C089804401C431AD06B68222B2B
:109A040013D14523DB004F48C65804980402A642EC
:109A14000BD24C4CA019526A272682554A4A049804
:109A2400A054E258521CE25003E0936908241C43FA
:109A3400946180200E46069006400A9830D00B9A16
:109A4400079B1A400C9B069C2340134328D03D4A95
:109A5400136884241C59212C14D11C4656342288A2
:109A6400002A0FD01A6802921A6D03921278019498
:109A7400029CA262039A521C1A65019B1A88521E08
:109A84001A8008E01A681368069CA34313601368DD
:109A940040241C4314602B4C23221201049BA35426
:109AA40040240C9B23405A425A41490600D5104693
:109AB40000280ED1254800210170059803681A6812
:109AC400A2431A6041670899296001F03BF92220FA
:109AD4006860A868002829D022236B60002F07D073
:109AE4000B98099901400C98089A104008431FD11B
:109AF400002E1BD00B99079801400C98069A104031
:109B0400084313D026200F4E0021315405981F46D8
:109B140003681A68A2431A6041670899296001F032
:109B240011F96F6023200001049931540DB0F0BD88
:109B340005980068816908220A4382610020A860B0
:109B44000DB0F0BDF8090020310200001E0A00200B
:109B5400F0B583B04521CB00C258052A3AD301930E
:109B64002721415C00910290044627341046951E3B
:109B74001C4900261C4F03E0761CAE4219460CD04B
:109B8400A35D4B400721C94302E01346491CF3D2AD
:109B94005A08DB07F9D07A40F7E7615D0219521ED3
:109BA400127812025118C91A4A1E9141401C4242AD
:109BB40042410A430298019B0CD10C49C98B009C79
:109BC4000A1B51425141002C00D10121002901D02E
:109BD400022103E0C218002101751160084603B098
:109BE400F0BDC046FFFF000001A00000340C0020BF
:109BF400F0B585B006468B208000049000273750CE
:109C04002720335CFF24204628303354009635182F
:109C1400314627310122284601F07EF90499711852
:109C240002914521C90071180391049632462632E7
:109C34000028214614D01449144B03E07F1C8742AA
:109C440021460CD0EC5D4C400721C94302E0344668
:109C5400491CF3D26608E407F9D05E40F7E7210A0D
:109C64002C542B1859700C211170811C029801601E
:109C7400049C20688AB22946FBF710FE0020039951
:109C84000860207505B0F0BDFFFF000001A00000D2
:109C9400F0B51E4C002B06D0E58B9D4203D08621E7
:109CA40081540B211BE04D790B791B025B191E4675
:109CB4007E3E7D27FF43BE4203D883218154032186
:109CC4000DE0CE788978090289195B181E468C3E0E
:109CD4008B27FF43BE4206D88321815402211018EA
:109CE4004170901CF0BD0326865486186D00757073
:109CF4004D00641985186678AE702678EE70A41C41
:109D0400921C491C9942F5D3901CF0BD340C0020E0
:109D1400F0B51D4C002B08D0E58B9D4205D0862163
:109D24008154531C02240B212AE0CB788D782D0218
:109D3400ED188B2D09D28D26B600059FBE19376804
:109D44007F5D022F07D0002F09D186218154531C37
:109D540002210C4614E076683688002EF5D06D009A
:109D640066190F7977704E796655062484548418E1
:109D7400A370002363700B79E370131D49790524E4
:0C9D8400C154A018F0BDC046340C0020F3
:109D9000F0B585B00490304D022401200390002BD3
:109DA00006D0E88B984203D00B26862310464BE062
:109DB0004F7908790002C01905467C3D7A23DE43BD
:109DC0009023B54202D2032610463DE00297CD789B
:109DD0008C780194240200956719C51928468C389F
:109DE0008A24E4430226A042104634462CD3164669
:109DF0008D2080000A9A13187800174A1418C91D7C
:109E000008E00878607048782070A41C891C7F1CCA
:109E1000AF420AD21868C05D0028F6D00228F0D1FF
:109E2000586800880028ECD1EFE7102032460499EA
:109E3000885588190099817001994170F01C05249A
:109E4000042103910023029E04990B540398801867
:0C9E50000E54A01805B0F0BD340C00202A
:109E5C0000B583B00D48416801221143416041684F
:109E6C00114002910299110702680A4302600068CE
:109E7C00084001900198F9F707FA0220F9F7FAF96E
:109E8C0003204002F9F708FA03B000BD3C10024071
:109E9C00FBF732F8054C064D0221204601F0A0F9E3
:109EAC000020294600F000FDF6E7C04600040050F3
:049EBC0015B90008CC
:109EC00000240749204600F0F5FC0649204600F032
:109ED000F1FC054C0221204601F088F9FAE7C04662
:0C9EE000C1BD0008C9BD0008000400500E
:109EEC0080B50248FBF70AFA80BDC046EC0F002093
:109EFC0080B50248FBF702FA80BDC046A00F0020D7
:109F0C0080B50248FBF7FAF980BDC0466811002005
:109F1C0080B50248FBF7F2F980BDC0461C11002049
:109F2C0080B50248FBF7EAF980BDC046D01000208E
:109F3C0080B50248FBF7E2F980BDC04684100020D2
:109F4C00B0B50446FBF7C0F920682349884227D0F6
:109F5C0022490968884232D0224988422ED0204CAE
:109F6C00216888422AD02049884231D01F49884232
:109F7C0024D1EA201F4900250D521F481F4A0260B8
:109F8C008D851F481F4901602046FBF79DF9012074
:109F9C00C043216808614D622046FBF75DF9B0BDF6
:109FAC00144C0125A585194800F0BCFAEA2025526D
:109FBC00114817490160124816490160B0BD0D489F
:109FCC000221818510480268002001219047B0BD14
:109FDC0007480121F1E7C04600100040A00F002007
:109FEC00681100200040014000480140004401403D
:109FFC00A4120020340C0020DC12002001000020F0
:10A00C002C130020118D00084C130020D5010020CA
:08A01C0031030020318D000822
:10A0240070B516490868164A13684340154C2268EF
:10A034001A40D5432560144C26681E406E402660A5
:10A044005A40324050400860024010490B681343A4
:10A054000B600C21014005D00D480268521E0260BD
:10A0640004D070BD0A480C49016070BD64220260CE
:10A07400084802680A43026070BDC0469812002076
:10A08400100C0050B0120020AC120020A0120020CE
:0CA09400A81200209C1200205F090000B0
:10A0A00004490968884304490A68104042400A602C
:0CA0B0007047C04698120020A01200204B
:10A0BC0005490A68104042400A6004490A68104089
:10A0CC0042400A607047C0469C120020A01200203B
:10A0DC0030B587B0154800248461E1430125AA07F7
:10A0EC0014C0046041608460069405940494019447
:10A0FC00083800F00FFD002801D0FEF763FD28039F
:10A10C0003900A4803A9FBF7ABF9002801D0FEF72E
:10A11C0059FD0294009405486946FBF741FA002862
:10A12C0001D0FEF74FFD07B030BDC04638100020FF
:10A13C0010B584B00E48002484610E49F9220E4BF0
:10A14C00036042608460C160029400F0E3FC00286C
:10A15C0001D0FEF737FD03940194054801A9FBF7E4
:10A16C001FFA002801D0FEF72DFD04B010BDC0462B
:0CA17C00EC0F0020FFF900000010004074
:10A1880010B584B00E48002484610E49F9220E4BA4
:10A19800036042608460C160029400F0BDFC002846
:10A1A80001D0FEF711FD03940194054801A9FBF7BE
:10A1B800F9F9002801D0FEF707FD04B010BDC0462C
:0CA1C800A00F0020FFF900000014004070
:10A1D40010B5094800218161084A6323084C0460D2
:10A1E40043608160C260016100F098FC002801D0E6
:10A1F400FEF7ECFC10BDC04668110020FFF900001A
:04A2040000200040F6
:10A2080010B588B0154800241549164A14C00460D2
:10A2180041608460C46004610794069405940294C4
:10A22800083800F079FC002801D0FEF7CDFC0120A9
:10A2380000030490094804A9FBF714F9002801D089
:10A24800FEF7C2FC03940194044801A9FBF7AAF99C
:10A25800002801D0FEF7B8FC08B010BD1C11002082
:08A26800FFFF0000004001406F
:10A2700010B509480021094A094B0A4C04604360A3
:10A280008160C26001614161816100F049FC002888
:10A2900001D0FEF79DFC10BDD0100020FFF900009A
:08A2A0005FEA000000440140E8
:10A2A80010B509480021094A094B0A4C046043606B
:10A2B8008160C26001614161816100F02DFC00286C
:10A2C80001D0FEF781FC10BD841000200F2700008C
:08A2D800FFF9000000480140FD
:10A2E00010B58EB0044601A8001D302100F0F6F92B
:10A2F00020683F4988421EDD3E49884230DC4049A3
:10A3000088423ED03F4988426FD10124A005019088
:10A3100001A8FAF70DFE002801D0FEF759FC200431
:10A320003B490A6802430A6009680140009114240D
:10A3300000210A4652E001218A0790422CD032497E
:10A34000884234D0314988424FD13148001F0168DA
:10A3500020221143016000681040009012243BE06D
:10A36000254988422ED0254988423ED101208004CB
:10A3700027490A6802430A600968014000911624CF
:10A380002AE00120C00322490A6802430A600968E2
:10A390000140009113241FE01D48001F02680A437A
:10A3A000026000680840009000980EB010BD184888
:10A3B000001F0168102211430160006810400090E6
:10A3C000112409E00120400411490A6802430A608F
:10A3D00009680140009115240321002200982046BD
:10A3E000F9F796FC2046F9F7B3FC0EB010BDC04655
:10A3F000FF1F0040FF43014000440140004801406E
:10A4000000200040004001400010004000140040C7
:04A4100040100240B6
:10A41400B0B51A4800210C22194B016241628162D5
:10A42400036001239C021B03E1256D0245608360E8
:10A43400C160046142618161C1610A460B46FBF758
:10A4440065FD002801D0FEF7C1FB0C480021FBF795
:10A45400A3FD002801D0FEF7B9FB08480021FBF753
:10A46400DBFD002801D0FEF7B1FB044800F0BDFC81
:10A47400002801D0FEF7AAFBB0BDC046F40D0020B1
:04A48400003801405B
:10A48800F0B595B0044603A808302C2100F022F955
:10A4980020682349884201D015B0F0BD02250495F3
:10A4A8000127039703A8FAF73FFD002801D0FEF71C
:10A4B8008BFBB8031B49CA680243CA60CA680240DA
:10A4C800109210980868384308600868384002906D
:10A4D80014970024139412941195092040021090A7
:10A4E800029805200195050710AE28463146FAF76F
:10A4F80043F814971394129701981190B80210908A
:10A5080028463146FAF738F81B2503212846224603
:10A51800F9F7FAFB2846F9F717FC15B0F0BDC04665
:08A5280000380140341002402C
:10A53000002801D0014908607047C046B8120020C9
:10A540004A0010D2520D03231B02FF33D21A0AD441
:10A5500052421F3209D4400DC90208430123DB07D0
:10A560001843D040704700207047D0177047C0464E
:10A5700042221201033A010007D002D4013A001826
:0CA58000FCD51205C30A4005991870476D
:10A58C00CA1751408B1A17D0C1174A4094464840FD
:10A59C00411A48081A0000E052008242FCD90020FF
:10A5AC0000E05208914200D3891A40419A42F8D1F6
:10A5BC0062465040801A704710B500F075F810BD17
:10A5CC000A0015D00300400800E052008242FCD97A
:10A5DC00002000E052089B1A06D340418A42F9D170
:10A5EC00704752089B18F8D200188A42F9D170476C
:08A5FC0010B500F059F810BD84
:10A6040038B504004D42FFF7DFFF4543611938BDFB
:10A61400002B09D1002907D110B51100FFF7F0FF75
:10A624000A000021002310BD70B400240125ED07A9
:10A63400002B07D1002905D0834203D21300002246
:10A644002C0000250026A419994200D1904212D969
:10A6540092185B4103D2EE076D086408F3E7DE0746
:10A664005B08520892190126F6079B1903E0DE07DE
:10A674005B0852089219801A994103D364416D41D1
:10A68400F5D30FE024196D410AD2DE075B085208A6
:10A69400921980185941F5D364416D41E7D301E023
:10A6A4008018594102000B002000290070BC70473B
:08A6B400002000217047C046A0
:10A6BC00411C02780130002AFBD1401A7047C04679
:10A6CC00002A03D0013A8B5C8354FBD17047C046FF
:10A6DC0000220B0011001A00002A02D0013A81540A
:04A6EC00FCD17047E6
:10A6F00003231048104A03614361104B8261C36118
:10A700008023DB000362002383624362C36202662C
:10A710000B4A53214266102282660367094AC366C8
:10A72000436700E0D17BC1540133013A102BF9D1CA
:10A730007047C0464C0D00206CA90008F8050020A9
:08A740000812002078A90008AE
:10A74800F8B54746CE46C568836804004068994610
:10A758005B1B80B50E00170098464019934207D935
:10A76800FFF7B0FFED19E560C0BCB946B046F8BDCB
:10A778001A00FFF7A7FF4B463100ED19ED1A2A0022
:0CA7880060684144FFF79EFFEDE7C0460B
:10A79400F8B54746CE46002380B588460700160024
:10A7A4009946C56884681BE0013B5B1B641BB4428B
:10A7B40000D934009C4200D91C007868220041462C
:10A7C4004019FFF781FF2D19A144A044361BBC6832
:10A7D400631B5A1E93415B421D40FD60002E06D050
:10A7E4003B699D42E0D3013B1B195B1BDEE74846F6
:08A7F400C0BCB946B046F8BD37
:10A7FC0070B50600431C5C00E418E00074001C4BB0
:10A80C00A419E400C0181B19DC6A1500012C06D031
:10A81C00022C1FD0002C10D00024200070BD9A6A8E
:10A82C005C6AA2421FD9013A121B2C00954200D936
:10A83C0014002200FFF782FFEFE79A6A5E6AB242C9
:10A84C000CD9013A961BB542E7D82A00FFF776FFE0
:10A85C002C00E2E7FFF798FF0400DEE71B6AD21832
:10A86C00013A961BEFE71B6AD218013A121BDCE780
:04A87C004C0D00205F
:10A88000F8B50B4B04001B780D001600002B0CD004
:10A89000EFF31087012181F3108832002900200096
:10A8A000FFF7ACFF87F31088F8BDFFF721FFEFE754
:04A8B0004C0D00202B
:10A8B400F8B5050008000C00FFF7FEFE0A4B060081
:10A8C4001B78002B0CD0EFF31087012181F3108843
:10A8D400320021002800FFF78FFF87F31088F8BDAE
:0CA8E400FFF704FFEFE7C0464C0D00201A
:10A8F000000000000400000002000000080000004A
:10A90000004B0000650001000100E80300000000AA
:10A91000000038004C0020034C04DD053F02B80065
:04A920000000000033
:08A924000A000000B80B00005E
:08A92C000100000064000000BE
:10A934000A000000B80B0000B80B0000B80B0000C0
:10A9440001000000640000006400000064000000D6
:10A95400034C206804348047FBE7FCF7CBFAFEE79E
:04A96400E0BD00084A
:04A96800D1300008E2
:09A96C005465726D696E616C00A6
:03A975003A200085
:10A9780000000000000054545220524547474553F8
:01A9880000CE
:10A989004465766963652049443A20756E6B6E6F3C
:03A99900776E00D6
:02A99C00FEE7D4
:02A99E00FEE7D2
:02A9A000FEE7D0
:02A9A200FEE7CE
:02A9A400FEE7CC
:02A9A600FEE7CA
:02A9A800FEE7C8
:02A9AA00FEE7C6
:02A9AC00FEE7C4
:02A9AE00FEE7C2
:02A9B000FEE7C0
:02A9B200FEE7BE
:02A9B400FEE7BC
:02A9B600FEE7BA
:02A9B800FEE7B8
:02A9BA00FEE7B6
:02A9BC00FEE7B4
:02A9BE00FEE7B2
:02A9C000FEE7B0
:02A9C200FEE7AE
:02A9C400FEE7AC
:02A9C600FEE7AA
:02A9C800FEE7A8
:06A9CA00F8F779FBC1E77C
:0AA9D00080B5806A00F055F880BDE4
:10A9DA0080B5806A816D40220A438265C16D042276
:0AA9EA000A43C26500F047F880BD83
:10A9F400F0B581B004465420205C012801D1022521
:10AA040038E026465436012737702046F8F780FD93
:10AA1400054600282CD1206D2521415C022911D145
:10AA2400F9F7EEFB00280DD00546A06D4021014347
:10AA3400A165206841681022914341602046F8F7DF
:10AA440095FD11E020684168102291434160204641
:10AA5400F8F78CFD0546002806D1FF200230A16DD1
:10AA64008143481CA06500252068C168B943C160C2
:0AAA740000203070284601B0F0BD4C
:02AA7E0070471F
:02AA800070471D
:02AA820070471B
:10AA840070B54279012A01D1022070BD02230371FD
:10AA940010240C4001221546A540046826682E4364
:10AAA4002660256800290ED01E468E401F214904C9
:10AAB4000D40B54202D161681943616000214171C2
:10AAC4000271084670BD3E210D40022D1346F2D09E
:02AAD400F4E7A5
:10AAD60010B581B00024009400680090002903D0CE
:10AAE60000981018143002E00098101808300090F2
:0AAAF60000980360002001B010BDBD
:10AB000010220A401F2191400068806B0840D0400D
:02AB100070478C
:0AAB120000690840411E88417047A9
:02AB1C00704780
:02AB1E0070477E
:10AB2000F0B581B0002823D0044605463C350746E1
:10AB30003E37064644366878002803D12870204600
:10AB4000FFF7CEFB0220687001CC2146FAF7F4FA39
:10AB50000120307138707870B870F8703871787181
:10AB600030707070B070F0706870002001B0F0BD8F
:06AB7000012001B0F0BD60
:02AB7600704726
:02AB7800704724
:02AB7A00704722
:02AB7C00704720
:02AB7E0070471E
:02AB800070471C
:02AB820070471A
:10AB840030B5816ACA070CD18A0714D44A071CD489
:10AB94000A0724D4CA062CD48A0634D44A063CD4E0
:10ABA4004CE00122520403685C689443C26A224365
:10ABB4005A608A07EAD50122120403685C68944348
:10ABC400026B22435A604A07E2D5012292040368C9
:10ABD4005C689443426B22435A600A07DAD5012227
:10ABE400D20303685C689443826B22435A60CA06AA
:10ABF400D2D50122120303689C689443C26B22439A
:10AC04009A608A06CAD50122520303689C68944359
:10AC1400026C22439A604A0610D501221305026889
:10AC240054689C43456C2C4354609D4206D10323D5
:10AC34005B0554689C43836C23435360090607D522
:10AC44000121C904026853688B43C06C18435060E7
:02AC540030BD11
:10AC5600F0B585B0049316460F4604460368D969D5
:10AC66003940C91B4A424A410020B24242D10290B1
:10AC76002146803101910A9D01210091C80203906D
:10AC860006E0D9693940C91B4A424A41B24230D12D
:10AC9600691CF6D0F8F7D9FA002D2DD00499401A80
:10ACA600A84229D8236819684907EAD5D9690398BB
:10ACB6000142E6D01862EFF31080009D85F31088FC
:10ACC6000D214901226813688B43136080F31088B5
:10ACD600EFF3108085F3108821688A68AA438A609A
:10ACE60080F310882020019A5060906010460C3046
:10ACF6001EE0029805B0F0BDEFF31080009D85F3CD
:10AD060010880D214901226813688B43136080F374
:10AD16001088EFF3108085F3108821688A68AA43AB
:10AD26008A6080F310882020019A5060104608300F
:0EAD36000021117020210160032005B0F0BD46
:02AD4400704756
:02AD4600704754
:02AD4800704752
:02AD4A00704750
:10AD4C0070B5026801465C318B88CC6A222C0DD11F
:10AD5C00526A1A40836D1A704A88521E4A80826D5C
:10AD6C00521C82654A88002A05D070BD9069082162
:10AD7C000143916170BDEFF31083012282F31088BF
:10AD8C000924640105682E68A6432E6083F310889D
:10AD9C00EFF3108382F310880468A5689543A560CF
:10ADAC0083F310882023CB6200230367C46E012C2D
:10ADBC0014D1C366EFF3108382F3108804682568FE
:10ADCC0010229543256083F310880368DC69E40640
:10ADDC0000D51A620988FFF7B0FF70BDFFF7AFFF0F
:02ADEC0070BD38
:10ADEE0030B58021415C012901D1022030BD0246DF
:10ADFE0080322421516001680B680C680125AC4338
:10AE0E000C606C07A3430B6000214166117020207B
:06AE1E005060084630BD43
:06AE2400F920C000704798
:10AE2A00F0B581B0002816D014460D460646FF2715
:10AE3A004E3701222846214600F0CBF93846F8F76A
:10AE4A0008FA00222846214600F0C3F93846F8F7E6
:0AAE5A0000FA761EEDD101B0F0BD44
:10AE6400F0B581B01D4614460F460646F8F7EEF9D4
:10AE74003A68AA420BD22368022B1CD005460999D2
:10AE84000898012B07D0002B03D101220BE00020EE
:10AE9400386001B0F0BD069B52009A5A3368EB1A31
:10AEA4009342F6D9002200F097F935602068401CDF
:10AEB400206001B0F0BD034607985100405A316844
:10AEC400591A8142E5D93360002020603868401C5B
:02AED400DEE7B7
:10AED600B0B582B01D4613460A4604460B200190C3
:10AEE600022B01D3022000E00120009020462946D3
:10AEF600FEF775FC2620002121548D208000069A3D
:10AF06002250A184E161218420181C34A171079983
:06AF1600416002B0B0BD75
:10AF1C00B0B582B04C78069D102C07D0062C0AD008
:10AF2C00032C0DD1FEF7B0FE02B0B0BD0095FEF7BC
:10AF3C0029FF02B0B0BD0095FEF7E6FE02B0B0BD31
:10AF4C0080214C408454801801214170901C02B027
:02AF5C00B0BD86
:02AF5E0070473A
:02AF6000704738
:10AF620008D1002806D1F54204D801D3002A01D124
:10AF72006D0D09D10020C143090DC904F0BDF9D1FD
:10AF82001242F7D1640DF5D00020C14349054908AA
:10AF9200A6E000206146F0BDF0B50127FF070E00D4
:10AFA2005E403E40B446BE0A4C18DD18F442D7D289
:10AFB200F542E4D2640DECD06D0DEAD06419C902F9
:10AFC2003943460DC0023143DB023B43DB0A10B476
:10AFD2008E4685B297B26F43140C6C433E0CA41993
:10AFE200260C2404BFB227439CB26C43A419190C4B
:10AFF2006943250CA4B249190D04090C6419000C0B
:10B0020095B245433E0C76193743BFB2360C150C48
:10B012004543AD19A6B2240CAD192E0437432E0CAC
:10B0220036199DB24543AD19ACB22E0C89191D0CCF
:10B0320045436D182E04290C3443704680B295B2F4
:10B0420045433E0C76193743BFB2360C150C4543C7
:10B05200AD19A6B2AD19240C2E0437432E0C3619A5
:10B062009DB24543AD19ACB22E0C89191D0C454356
:10B072006D182E043443290C75462D0C90B268438A
:10B082003E0C80190604BFB23E43070CA0B23F1823
:10B09200120C6A43D019020C80B2240CA4189AB282
:10B0A2006A43121914042043120C89181B0C6B43B7
:10B0B200C91810BC01273D05294203D1B6194041E8
:10B0C2004941013CFF077D0D013D641B0BDB6D0017
:10B0D200AC4209DA240500254208BE4168416141BB
:0AB0E20066463143F0BD54E74EE727
:10B0EC00B0B504465420205C012801D10220B0BD2B
:10B0FC0025465435012028702046F8F705FA00281B
:10B10C000BD12046F8F72EFA002806D1FF2002308A
:10B11C00A16D8143481CA065002000212970B0BDA1
:10B12C00B0B50146806A836D826D5024234206D0EF
:10B13C00D20610D4006D426B08469047B0BD012179
:10B14C004B021A4382650268D3681B059B0F05D01E
:10B15C00FFF78FFCB0BDFFF78DFCB0BD837E002BDD
:10B16C00F6D113681B07F3D593685B070AD4034623
:10B17C00583354680C25AC435460FF2402341A68CD
:10B18C00A24306E0826D20231343836503465C33A0
:0CB19C00C26D0A431A60FFF76CFCB0BDE6
:0CB1A8000068B42141587F200840704727
:10B1B40010B500280ED004460079002803D1607130
:10B1C4002046FBF783FB022020710020206101212F
:08B1D400217110BD012010BD26
:10B1DC00002A02D0182281507047282281507047D3
:10B1EC0042690B4693430A401104C91881617047A8
:10B1FC0030B584214158212904D1014656318A8A1F
:10B20C00002A03D130BD521E1304FBD00B88002B37
:10B21C000CD00368DC692406F5D5046D25789D6295
:10B22C00631C03650B885B1E0B80ECE7EFF310814E
:10B23C00012282F31088D3050468A5689D43A5609C
:10B24C0081F31088EFF3108182F310880068026894
:0CB25C0040231343036081F3108830BDD1
:10B2680030B58421415821290DD1014656310A882B
:10B27800002A09D00268036D1C7894625A1C026582
:10B288000888401E088030BDEFF31081012282F348
:10B29800108803681C688025AC431C6081F3108803
:10B2A800EFF3108182F3108800680268402313438B
:08B2B800036081F3108830BD32
:10B2C00070B5026801465C318B88CC6A222C0CD1A7
:10B2D000526A1340826D13804B885B1E4B80921C18
:10B2E00082654A88002A05D070BD90690821014313
:10B2F000916170BDEFF31083012282F3108809245D
:10B30000640105682E68A6432E6083F31088EFF36E
:10B31000108382F310880468A5689543A56083F3C1
:10B3200010882023CB6200230367C46E012C14D144
:10B33000C366EFF3108382F3108804682568102237
:10B340009543256083F310880368DC69E40600D523
:10B350001A620988FFF7F7FC70BDFFF7F6FC70BDB5
:10B3600010B5044642688368581C904203D91846B9
:10B37000904209D010BD2268D154A060E168491CF8
:10B38000E16062689042F5D121682069FFF778FAA0
:10B39000A168884202D10020A06010BD0020C043F7
:04B3A000E06010BD9C
:10B3A40082B000B581B00292039302AA00926A4669
:0CB3B400FAF772FE01B002BC02B00847BC
:04B3C000007D704755
:10B3C400010002000400060008000A000C0010003E
:08B3D400200040008000000190
:10B3DC00547279696E6720746F2072657374617230
:03B3EC00742E00BC
:10B3EF0043616E6E6F742072656164207374617453
:10B3FF0069737463616C20646174612066726F6D30
:0FB40F0020464C415348206D656D6F72792100C6
:10B41E004144432063616C6962726174696F6E208E
:07B42E006572726F722100CC
:10B435005374617274696E6720566563746F722008
:10B445005461626C6520636F7079696E67206672FE
:10B455006F6D20464C41534820746F2052414D2E4C
:03B465002E2E0088
:10B468004D6F646520302069732073656C65637463
:10B4780065642E204175746F2D7265636F6E6E65FD
:0BB488006374206973204F46462E00BD
:10B493004D6F646520312069732073656C65637437
:10B4A30065642E204175746F2D7265636F6E6E65D2
:0BB4B3006374206973204F46462E0092
:10B4BE004D6F646520322069732073656C6563740B
:10B4CE0065642E204175746F2D7265636F6E6E65A7
:0BB4DE006374206973204F46462E0067
:10B4E9004D6F646520332069732073656C656374DF
:10B4F90065642E204175746F2D7265636F6E6E657C
:0BB509006374206973204F46462E003B
:10B514004D6F646520342069732073656C656374B2
:10B5240065642E204175746F2D7265636F6E6E6550
:0BB534006374206973204F46462E0010
:10B53F004D6F646520352069732073656C65637486
:10B54F0065642E204175746F2D7265636F6E6E6525
:0BB55F006374206973204F46462E00E5
:10B56A00555020627574746F6E206973206C6F6E0B
:0BB57A00672D707265737365642E000E
:0BB5850056613A20253664206D560008
:0BB5900056623A20253664206D5600FC
:0BB59B004441435F413A202534640026
:0BB5A6004441435F423A20253464001A
:03B5B1004F5000F8
:03B5B400434C0005
:03B5B7004241000E
:03B5BA004142000B
:03B5BD00257300F3
:03B5C0004F5400E5
:03B5C3004F4300F3
:03B5C6004F4C00E7
:03B5C9004C4200F1
:10B5CC0043757272656E742063616C6C6962726132
:10B5DC0074696F6E2073657175656E636520737425
:07B5EC0061727465642E001A
:10B5F300095B2534645D2053616D706C656420764E
:0BB60300616C75653A202534640A0074
:0BB60E0048414C206572726F722100F1
:10B6190053415645204C4F434B2D4B455920434FE1
:07B629004D4D414E442E007F
:10B6300043616E6E6F7420726573746F72652064FF
:10B64000656661756C742073657474696E677320C8
:10B6500066726F6D20464C415348206D656D6F7268
:03B660007921004D
:02B663000A00DB
:10B665004465766963652049443A2053544D333225
:10B6750047304231206F722053544D3332473043A7
:02B68500310092
:10B687004465766963652049443A2053544D333203
:10B6970047303731206F722053544D33324730389B
:02B6A700310070
:10B6A9004465766963652049443A2053544D3332E1
:10B6B90047303531206F722053544D33324730367D
:02B6C90031004E
:10B6CB004465766963652049443A2053544D3332BF
:10B6DB0047303331206F722053544D33324730345F
:02B6EB0031002C
:10B6ED004672656520737061636520666F722063B5
:10B6FD006F66696775726174696F6E20696E206619
:10B70D00616B6520454550524F4D3A20257520629D
:06B71D00797465730A0057
:10B723004D41585F504F535349424C455F4449463E
:10B73300465F544F5F4D4541535552453A20257559
:02B743000A00FA
:10B7450043616E6E6F74207374617274204144435B
:0EB7550020696E20444D41206D6F6465210017
:10B7630043616E6E6F7420636F70792056656374E6
:10B773006F72205461626C652066726F6D20464C57
:10B7830041534820746F2052414D2120444D4120A4
:0EB793006973206E6F74207265616479210005
:10B7A10043616E6E6F742066696E69736820636FA2
:10B7B1007079696E6720566563746F722054616297
:10B7C1006C652066726F6D20464C41534820746F42
:06B7D1002052414D210051
:10B7D7004D6F646520302069732073656C656374F1
:10B7E70065642E204175746F2D7265636F6E6E658B
:0AB7F7006374206973204F4E2E008A
:10B801004D6F646520312069732073656C656374C5
:10B8110065642E204175746F2D7265636F6E6E6560
:0AB821006374206973204F4E2E005F
:10B82B004D6F646520322069732073656C6563749A
:10B83B0065642E204175746F2D7265636F6E6E6536
:0AB84B006374206973204F4E2E0035
:10B855004D6F646520332069732073656C6563746F
:10B8650065642E204175746F2D7265636F6E6E650C
:0AB875006374206973204F4E2E000B
:10B87F004D6F646520342069732073656C65637444
:10B88F0065642E204175746F2D7265636F6E6E65E2
:0AB89F006374206973204F4E2E00E1
:10B8A9004D6F646520352069732073656C65637419
:10B8B90065642E204175746F2D7265636F6E6E65B8
:0AB8C9006374206973204F4E2E00B7
:10B8D300555020627574746F6E20697320707265A1
:06B8E300737365642E0082
:02B8E9004E000F
:06B8EB00523A2025730013
:02B8F1000A004B
:10B8F30043616E6E6F742073617665206461746159
:10B9030020696E20464C415348206D656D6F7279F6
:02B91300210011
:0EB915004E4D49204552524F522121210A0029
:05B923004D41494E00FA
:10B9280043616E6E6F742073746172742054494D54
:05B93800455232210020
:05B93D001B5B324A0013
:10B9420050726F6772616D20737461727465642ED8
:01B9520000F4
:10B9530043505520467265713A20257520487A0A6E
:01B9630000E3
:10B9640043616E6E6F74207265616420636F6E66EE
:10B97400696775726174696F6E2066726F6D2046B7
:0DB984004C415348206D656D6F72792100B4
:10B99100257325733A204144432043616C696272E7
:10B9A1006174696F6E2076616C75653A2025750A40
:01B9B1000095
:10B9B20043616E6E6F742073746F70204144432133
:01B9C2000084
:10B9C30025733A204441432043616C696272617478
:10B9D300696F6E2076616C756520666F722063688F
:0DB9E300616E6E656C20313A2025750A00FA
:10B9F00025733A204441432043616C69627261744B
:10BA0000696F6E2076616C756520666F7220636861
:0DBA1000616E6E656C20323A2025750A00CB
:10BA1D0049742069732074696D6520746F2073619A
:10BA2D00766520737461746973746963616C2064E5
:10BA3D0061746120696E20466C617368206D656D5F
:05BA4D006F72792E006C
:10BA5200496C6C6567616C204D6F64652069732069
:10BA620073656C65637465642E2044656661756CEC
:10BA720074204D6F646520342069732073656C6592
:10BA8200637465642E204175746F2D7265636F6EE9
:0DBA92006E656374206973204F46462E00D8
:05BA9F00257325730072
:09BAA400493A20253564204100D7
:09BAAD004F56503A202531730078
:09BAB6004C56503A202531730072
:0DBABF00543A202532642E256420B0430047
:10BACC00095B2534645D2053616D706C6564207670
:10BADC00616C7565733A20492B203D202536752005
:0DBAEC00202020492D203D202536750A0020
:10BAF90009094F66667365742076616C7565733ADA
:10BB090020492B203D20257520202020492D203D2E
:05BB19002025750A0063
:10BB1E0009094F66667365742076616C75653A2007
:05BB2E002534640A004B
:10BB3300556E6B6E6F776E20636F6D6D616E6421F2
:01BB43000001
:0DBB44005553415254206572726F722100FA
:08BB51000101010307010000DE
:08BB59000804020408010101C7
:10BB61003031323334353637383941424344454632
:08BB71001B5B323B33326D0017
:08BB79001B5B323B33336D000E
:08BB81001B5B323B33316D0008
:10BB890025733A205265766973696F6E206E756DFB
:0CBB99006265723A2030782534580A00AA
:10BBA5004672656520737061636520666F722073E8
:10BBB50074617469737469637320696E2066616B5F
:10BBC5006520454550524F4D3A20257520627974C0
:04BBD50065730A008A
:10BBD900435055207370656564206973206E6F74D6
:08BBE9002036344D487A21009A
:10BBF100466972737420737461727421205772697B
:10BC010074696E672064656661756C7420636F6E1C
:0CBC110066696775726174696F6E2100CE
:08BC1D001B5B313B33326D006B
:10BC2500566563746F72205461626C652068617338
:10BC3500206265656E20636F706965642066726F4A
:10BC45006D20464C41534820746F2052414D2E00C3
:10BC5500496C6C6567616C204D6F64652069732064
:10BC650073656C65637465642E2044656661756CE7
:10BC750074204D6F646520342069732073656C658D
:10BC8500637465642E204175746F2D7265636F6EE4
:0CBC95006E656374206973204F4E2E0012
:10BCA100444F574E20627574746F6E206973207013
:08BCB1007265737365642E00D7
:08BCB9001B5B323B33306D00D0
:08BCC1002573207C202573008F
:0CBCC9005661623A20253464206D56005C
:0CBCD5005662623A20253564206D56004E
:10BCE1001B5B323B33316D591B5B313B33326D0092
:08BCF1001B5B313B33316D0098
:08BCF9001B5B313B33366D008B
:08BD0100434847202D203100CA
:08BD0900434847202D203000C3
:10BD11000909566F6C746167652D64726F702041FB
:10BD210044432076616C75653A202535642E0A00FE
:10BD310009090946696E616C20766F6C74616765EB
:10BD41002D64726F70204144432076616C75653AB1
:10BD5100202534752E2046696E616C20766F6C74D7
:10BD61006167652D64726F702076616C75653A202C
:08BD7100253375206D560A0010
:10BD790043616E6E6F742073617665206E657720FE
:10BD8900534E20696E20464C415348206D656D6FB6
:04BD9900727921009A
:10BD9D0043616E6E6F742073746172742054494DDB
:10BDAD00313720696E20495352206D6F6465210033
:04BDBD004D4F4400A2
:08BDC1001B5B313B33316D00C7
:10BDC900486172646661756C74204552524F522104
:04BDD90021210A001A
:03BDDD00FFFFFF66
:10BDE00059E30008E70400207E0E000059E3000834
:10BDF000661300200300000059E300086A130020C6
:10BE00000300000059E300086E1300200300000047
:10BE100059E30008721300200300000059E30008F2
:10BE2000781300200100000059E300087C13002073
:10BE30000100000059E30008801300200100000009
:10BE400059E30008821300200C0000006BE3000897
:10BE50000000002070BE0008E70400006BE300084B
:10BE60000060002057C30008002000005FA9000800
:10BE700006480068C16A0E2900D90F39026B81603B
:10BE80000E2A00D90F3A42617047C046F4110020D3
:10BE900006480068C26A06498A4200D20F32036B24
:10BEA00082608B4200D20F3343617047F41100204F
:10BEB000F10F000006480068C16A0E2900D90F3949
:10BEC000026B81600E2A00D90F3A42617047C0466A
:10BED000F411002006480068C26A06498A4200D26E
:10BEE0000F32036B82608B4200D20F334361704785
:10BEF000F4110020F10F000006480068C16A0E2905
:10BF000000D90F39026B81600E2A00D90F3A4261C5
:10BF10007047C046F411002006480068C26A06490E
:10BF20008A4200D20F32036B82608B4200D20F3301
:10BF300043617047F4110020F10F0000F0B517487D
:10BF40000068C16A3A22164B9C5E164D2A68121987
:10BF5000154EB242154F03DA0E2912D8002311E014
:10BF600001230022B9421F4600D317462D682C1921
:10BF7000B44200DC13463B400F220C4F002B05D18E
:10BF800005E001230E22D243002B00D089188160E6
:10BF9000016BB94200D20F314161F0BDF4110020B4
:10BFA000340C00207412002098090000F10F0000EA
:10BFB000F0B517480068016B3A22164B9C5E164D8F
:10BFC0002A681219154EB242154F03DAB9421AD334
:10BFD000002319E0012300220E291F4600D817462E
:10BFE0002D682C19B44200DC13463B400E22D2438C
:10BFF0000B4F002B00D089184161C16AB94200D2B1
:10C000000F318160F0BD01230F22002BF3D1F3E744
:10C01000F4110020340C0020741200206606000089
:10C02000F10F000006480068C16A0E2900D90F39D7
:10C03000026B81600E2A00D90F3A42617047C046F8
:10C04000F411002006480068C26A06498A4200D2FC
:10C050000F32036B82608B4200D20F334361704713
:10C06000F4110020F10F00007047010180B500F0CD
:10C0700077F880BD10B5154C208915490880154802
:10C0800000688047A088144908606089134A1060DE
:10C090001348036802241C4304600868116888423E
:10C0A00000DC084640210F4A515E88420AD30E49FF
:10C0B0000A68101808600D490968884205D90C48BB
:10C0C0000068804708480021016010BD82130020ED
:10C0D00074120020DC120020781200207C12002054
:10C0E00004000240340C0020341300201C04002003
:10C0F000F812002080B500F03BF80C2000F040F86A
:10C100000B480C4901600C480068002800D080BD35
:10C110004120800009490A5A521C0A52084801214C
:10C12000016008480160084800680849086080BD4F
:10C13000DC120020F901002080120020340C0020C5
:10C1400084120020701200206812002018040020C1
:10C1500080B5024800F01CF880BDC046F40D0020F8
:10C1600008B4024B9C4608BC6047C0463932000800
:10C1700008B4024B9C4608BC6047C046058C0008CA
:10C1800008B4024B9C4608BC6047C046693D0008A5
:10C1900008B4024B9C4608BC6047C046059900089D
:10C1A00010B525480168022910D0012932D0002994
:10C1B0002FD122490A68002191605161204A1368F9
:10C1C0005C1C1460102B24DB116030E01B490A68F2
:10C1D0000021916051611A4A13685C1C1460002BA5
:10C1E00017D40160116017480268531C0360164B96
:10C1F0009A420EDB01600924204600F02FF8134814
:10C200000068002800D1124812490860204600F05A
:10C210002DF810BD094909680F4A8A604A6108492A
:10C220000A68531C0B60002AF3D400220A600168DC
:10C23000491C016010BDC046CC120020F411002042
:10C24000D4120020D01200203F060000B8120020B7
:10C25000F9010020DC120020FF0F000008B4024B9F
:10C260009C4608BC6047C046693D000808B4024BC4
:10C270009C4608BC6047C046513D000804000000D1
:10C28000FFFFFFFFC0E0FFFFC0E0FFFFFFFFFFFF7A
:10C290000024F40001000000FFFFFFFF0100000088
:10C2A000FFFFFFFF01000000FFFFFFFF0100000094
:10C2B00000B80B00020000000100000004000000B4
:10C2C000010000000200000001000000000000006A
:10C2D000020200000000000202020202010000004F
:10C2E0000000000000000000000101010001010049
:10C2F0000100020201010000000000000000000037
:10C30000000000000000000000000000000000002D
:10C31000000000000000000000000000000000001D
:10C32000000000000000000000000000000000000D
:10C3300000000000000000000001010101000101F7
:10C3400000000001010101000000000000000000E9
:10C3500000000000000000CDCDCDCDCDCDCDCDCDA8
:10C36000CDCDCDCDCDCDCDCDCDCDCDCDCDCDCDCDFD
:10C37000CDCDCDCDCDCDCDCDCDCDCDCDCDCDCDCDED
:10C38000CDCDCDCDCDCDCDCDCDCDCDCDCDCDCDCDDD
:10C39000CDCDCDCDCDCDCDCDCDCDCDCDCDCDCDCDCD
:08E35000CDCDCDCDCDCDCD002A
:10E35800206861680834002200E042540139FCD585
:02E368007047FC
:10E36A0020686168A2680C3401E08B5C8354013A2E
:04E37A00FBD5704718
:10E37E00FFFFFFFFFFFFFFFFFFFFFFFFFFFFFFFF9F
:10E38E00FFFFFFFFFFFFFFFFFFFFFFFFFFFFFFFF8F
:10E39E00FFFFFFFFFFFFFFFFFFFFFFFFFFFFFFFF7F
:10E3AE00FFFFFFFFFFFFFFFFFFFFFFFFFFFFFFFF6F
:02FFFE00FFFF03
:020000040801F1
:10000000FFFFFFFFFFFFFFFFFFFFFFFFFFFFFFFF00
:10001000FFFFFFFFFFFFFFFFFFFFFFFFFFFFFFFFF0
:10002000FFFFFFFFFFFFFFFFFFFFFFFFFFFFFFFFE0
:10003000FFFFFFFFFFFFFFFFFFFFFFFFFFFFFFFFD0
:04EFFC00F6EB1865B3
:040000050800A9CB7B
:00000001FF
